:1066AC000000090200000301FA0400FA0500030AC5
:1066BC000A5A0B001E0C00FA0D00030E00040F0109
:1066CC0064100096120132130AFA14020217010A1E
:1066DC001801FA1905321A010A1B01FA1C05321F9E
:1066EC00FFFF20FFFF23011E2400642A00FA2B0069
:1066FC00FA2C50782D003D2E004630006432507834
:10670C003300003432FA35016436016437015038F5
:10671C000A643C00643E003C3F000140FFFF411412
:10672C0050420A5A430AC84405324500B44600FA9E
:10673C004C00FA500808510596520A32530B465435
:10674C000A96570546590A465A32FA5B010A5C0A00
:10675C00325E000A5F00FE64011167FFFF6A0A3CAB
:10676C006B00006C32967300007400007801327973
:10677C0001327E00647FFFFF80FFFF8100008400F8
:10678C00648A00019D0A969E00019FFFFFA0FFFFF7
:10679C00A2000AA3FFFFA4FFFFA5FFFFA6FFFFA710
:1067AC00FFFFA8FFFFA9FFFF0101241502022F0024
:1067BC003C4701484802035602024EFFFF580002B4
:1067CC0061FFFF6600028500AF8600018700FA8931
:1067DC000107990008A100FAFAFAFA01012415023E
:1067EC00022F1E3C4701484802035602024EFFFF8F
:1067FC0058000261FFFF6600028500AF860001872A
:10680C0000FA890107990000A10000FAFAFA006564
:10681C00006F00790083008D009700A100AC00B6DA
:10682C0000C000CA00D400DE00E800F2005800608E
:10683C00006800700078008000880090009800A02C
:10684C0000A800B000B800C100C800D000D800DF1C
:10685C0000E600EE00F600410047004D00530059E1
:10686C00005F0065006C00710077007D008300897B
:10687C00008F0095009B00A200A700AC00B200B9ED
:10688C0000C000C500CA00D200D500DD00E100E761
:02689C0000EF0B
:10331000900898E0900124F0900899E0900093F0D4
:1033200090089AE09000B3F090089BE09000DCF0E9
:1033300090089CE0900088F090089DE09000CEF00E
:1033400090089EE09000ECF090089FE09000C0F0A4
:103350009008A0E09000DEF09008A1E090010EF04F
:103360009008A2E0900172F09008A3E0900173F041
:103370009008A4E0900174F0900172E0700C90014C
:1033800073E07006900174E060028004C221800244
:10339000D221743390015DF0743690015EF0742D8B
:1033A00090015FF07431900160F0742D900161F034
:1033B0007431900162F07420900163F0744E9001BA
:1033C00064F07469900165F07473900166F0746143
:1033D000900167F0746E900168F07420900169F0BC
:1033E000745690016AF0743890016BF02290089046
:1033F000E0FEA3E0FF7408D39F74019E400C90662A
:10340000AC120048E493F599802F900061E0D394CA
:10341000054014900890E0FEA3E0FF9066AC120017
:1034200048E493F5998012900890E0FEA3E0FF90A5
:1034300066DF120048E493F5999008901269BE90F7
:103440000890E0FEA3E0FFEFB43B07EEB401037584
:103450004C002285F97285FA737E017F00E57312B4
:1034600069B0E5722FFF50010E8E598F5A90001DE2
:10347000E0FCA3E0FDEF2DFDEE3CFC8C5B8D5C22BF
:1034800075A71085F97285FA737E017F00E57312C6
:1034900069B0E5722FFF50010E8E598F5A90001DB2
:1034A000E0FCA3E0FDEF2DFDEE3CFC8C5B8D5C228F
:1034B000E55CF5FBE55BF5FCD29322E55CF5E9E51F
:1034C0005BF5EAD29422E55CF5EBE55BF5ECD29195
:1034D00022E55CF5EDE55BF5EED29222E55CF5FBCD
:1034E000E55BF5FCD28722E55CF5E9E55BF5EAD220
:1034F0009022E55CF5EBE55BF5ECE5B54410F5B540
:1035000022E55CF5EDE55BF5EEE5B54420F5B52289
:10351000AE59AF5A740A8E048F05FF1269A08C5BF6
:103520008D5CAE59AF5A740A8E048F05FF1269CBB9
:103530008C598D5AE55A45596013740AC3955AFF40
:10354000E49559FE8E598F5A785B126A03E572A88A
:103550005BB80015D3955C4010E572C3955CFFE441
:10356000955BFE8E5B8F5C8010E5722424C3955CB6
:10357000FFE4955BFE8E5B8F5CAE5BAF5C74126F9D
:103580004E600674246F4E700A785B126A0B757277
:103590000180037572002290009AE0B40104C20613
:1035A0008002D20690009BE0B40104C2078002D2E0
:1035B000079000D8E075F0E1A4FFAEF0740A8E0425
:1035C0008F05FF1269A0900888ECF0A3EDF0740756
:1035D0008C068D071269B074038E048F05FF126983
:1035E000A0900019ECF0A3EDF07E017F0090009612
:1035F000E01269B09000D9E08E048F05FF1269A037
:10360000740AFF1269A08D5F9000E2E075F0E1A4FA
:10361000FFAEF0740A8E048F05FF1269A090088C2B
:10362000ECF0A3EDF09000E4E060139000E4E0F52E
:10363000F0741684FF7E00EF9008B4F08006746486
:103640009008B4F09000DAE0900078F0900126E065
:10365000900080F0900128E0FE9000D6E08E008877
:10366000F0A4FFAEF0EF9008BCF0900124E09008C9
:1036700098F09000B3E090089AF09000DCE0900899
:103680009BF0900088E090089CF090010EE090087C
:10369000A1F0900172E09008A2F0900173E0900810
:1036A000A3F0900174E09008A4F0A221B34016901A
:1036B0000172E0700C900173E07006900174E0609C
:1036C000028002C221900172E0B4300F900173E0D9
:1036D000B44708900174E0643B60028004D2228009
:1036E00002C22274E3900077F09000C3E0B40B08AC
:1036F00074E3900077F0805A9000C3E0B419129000
:1037000000D9E090680512008CE493900077F08077
:10371000419000C3E0B41E129000D9E090682312DB
:10372000008CE493900077F080289000C3E0B428E8
:10373000129000D9E090684D12008CE493900077CD
:10374000F0800F9000C3E0B446089000BAE090000B
:1037500077F090007BE0FE9000C0E0B5063390006B
:103760007CE0FE9000ECE0B5062790007DE0FE9046
:1037700000DEE0B5061B90007FE0FE900093E0B510
:10378000060F90007EE0FE9000CEE06E70030239DE
:103790006C9000CEE0640360069000ECE06008747A
:1037A0000390010FF08006740790010FF09000EC79
:1037B000E0B402089000CEE064036002800674006A
:1037C0009000ECF0900093E0B4020674009000DEEC
:1037D000F0900093E0B4030674009000EBF09000CA
:1037E000DEE0D39401402774009000A8F0741B9091
:1037F0000111F074009006D0F074009006D1F090A2
:1038000000C0E0B4020674019000C0F08033900064
:10381000C0E0B4021A741B9000A8F074009001116B
:10382000F074009006D0F074009006D1F08012740D
:10383000009000A8F07400900111F0741B9006D065
:10384000F09000CEE0B403089000ECE06402600267
:10385000800674009000ECF09000ECE0B401089059
:1038600000CEE0640360028026741C900112F074A4
:10387000009000A7F074009006D4F074009006D574
:10388000F09000C0E0600674009000C0F0803290BC
:1038900000C0E0601A741C9000A7F0740090011240
:1038A000F074009006D4F074009006D5F080127485
:1038B00000900112F074009000A7F0741C9006D4E0
:1038C000F09000CEE0B402069000ECE06002801AB6
:1038D00074059006D8F074069006DCF07407900624
:1038E000E0F074089006E4F0803074009006D8F0A0
:1038F00074009006D9F074009006DCF07400900615
:10390000DDF074009006E0F074009006E1F07400C1
:103910009006E4F074009006E5F0D2209000C0E03C
:1039200090007BF09000ECE090007CF09000DEE0F6
:1039300090007DF09000CEE090007EF0900093E04B
:1039400090007FF0900093E0900899F09000CEE016
:1039500090089DF09000ECE090089EF09000C0E090
:1039600090089FF09000DEE09008A0F09000F6E054
:10397000B40117900029740FF0A374FFF090002B8E
:10398000E4F0A3F074029000F6F09000F6E0B403C7
:103990004190002BE0FEA3E0FF900029E0FCA3E0B3
:1039A000FD1269FB74101269B07408120039EF90AF
:1039B0000074F0EF700674FF900074F074009000D3
:1039C000F6F090002AE0900075F0900029E0900059
:1039D00076F0900087E0900084F0900086E0900000
:1039E00083F09000B5E0C3941E50569000B5E0F40B
:1039F00004241E900085F0900085E075F00A84FF95
:103A00007E008F72900085E075F00A84ADF07C0036
:103A10008D73900083E0D39573400D900083E0C3D5
:103A20009573900083F0800F900083E0240AC39583
:103A300073900083F00572900084E02572900084FA
:103A4000F0900084E090004DF090004DE0D394247D
:103A5000400B90004DE0C3942490004DF090004D39
:103A6000E0240990004EF090004DE0241290004FA9
:103A7000F090004DE0241B900050F090004EE0D3F9
:103A80009424400B90004EE0C3942490004EF0909C
:103A9000004FE0D39424400B90004FE0C394249057
:103AA000004FF0900050E0D39424400B900050E081
:103AB000C39424900050F0900055E4F090004DE045
:103AC0006412600790004DE0B4241B90005574010F
:103AD000F090004DE0B41208741190004DF0800693
:103AE00090004D7401F0900056E4F090004EE064B8
:103AF00012600790004EE0B4241B9000567401F051
:103B000090004EE0B41208741190004EF0800690C0
:103B1000004E7401F0900057E4F090004FE0641202
:103B2000600790004FE0B4241B9000577401F090A0
:103B3000004FE0B41208741190004FF0800690001E
:103B40004F7401F0900058E4F0900050E06412606F
:103B500007900050E0B4241B9000587401F09000CE
:103B600050E0B412087411900050F080069000509C
:103B70007401F0900087E0FE9000EAE02E90005A79
:103B8000F090005AE06412600790005AE0B42406F6
:103B900090005AE004F090005AE0D39424400B9037
:103BA000005AE0C3942490005AF090005AE0D39455
:103BB00012400D90005AE0C3941290005BF0800A0E
:103BC00090005AE0241290005BF07550129000CDE6
:103BD000E0900051F0900051E075F00984AFF07E64
:103BE00000EF4E7006900051E004F0900051E0B4F8
:103BF00049069000517401F0900051E0D3942440A4
:103C00000F900051E0C39424900051F0D21B800229
:103C1000C21B900051E02409900052F0900051E046
:103C20002412900053F0900051E0241B900054F0B7
:103C3000900052E0D39424400B900052E0C39424AF
:103C4000900052F0900053E0D39424400B90005326
:103C5000E0C39424900053F0900054E0D3942440A7
:103C60000B900054E0C39424900054F022C293C2FD
:103C700094C291C292C287C290E5B554EFF5B5E502
:103C8000B554DFF5B5C296C295C2A0C297C2A2C212
:103C9000A1E5B554BFF5B5E5B5547FF5B5E5B55427
:103CA000FBF5B5C208755D469000D0E07005756CF7
:103CB000028003756C0375540075530090001074F6
:103CC000FFF0A374DCF0C20FC211C213C21574C896
:103CD00090003DF074C8900041F074C8900045F029
:103CE00074C8900049F0755200755100C2037545C3
:103CF00000E56EB40903756E0075620090001FE464
:103D0000F0A3F0756F10C20BC20CC20DC20EC2023E
:103D1000755600755500900012E4F0A3F090001461
:103D2000E4F0A3F0C226755800755700900092E0A9
:103D300075F032A4FFAEF0900027EEF0A3EFF09004
:103D40000081E4F0900082E4F0C223C21AC21BC2D8
:103D50001C22755A00755900AE59AF5A7408C39F9A
:103D600074019E5003023E109066AC120048E4932A
:103D70009000861269E10FBF00010EE0FC9066AC76
:103D8000120048ECFEE493FFEEC39F5026AE59AFFD
:103D90005A0FBF00010E9066AC120048AE59AF5AE0
:103DA000E493FC9066AC120048E49390008612699C
:103DB000E1ECF0AE59AF5A9066AC120048E4939033
:103DC00000861269E1E0FC9066AE120048ECFCE46B
:103DD00093FDECD39D40199066AE120048E493FC2D
:103DE0009066AC120048E4939000861269E1ECF012
:103DF000AE59AF5A74022FFF50010E8E598F5A7868
:103E00005A740126F6500418E436F64003023D5871
:103E100022755A00755900AE59AF5A7433BE00036B
:103E20009F5003023EDE9067B4120048E493900076
:103E3000861269E10FBF00010EE0FC9067B412002A
:103E400048ECFEE493FFEEC39F5026AE59AF5A0FE5
:103E5000BF00010E9067B4120048AE59AF5AE49308
:103E6000FC9067B4120048E4939000861269E1EC7C
:103E7000F0AE59AF5A9067B4120048E493900086B0
:103E80001269E1E0FC9067B6120048ECFCE493FD97
:103E9000ECD39D40199067B6120048E493FC9067FC
:103EA000B4120048E4939000861269E1ECF0AE5938
:103EB000AF5A742D6F4E7006755A33755900AE594E
:103EC000AF5A74022FFF50010E8E598F5A785A74D0
:103ED0000126F6500418E436F64003023E17227518
:103EE0005A00755900AE59AF5A7433BE00039F5043
:103EF00003023FAC9067E7120048E49390008612FB
:103F000069E10FBF00010EE0FC9067E7120048EC8A
:103F1000FEE493FFEEC39F5026AE59AF5A0FBF0089
:103F2000010E9067E7120048AE59AF5AE493FC9037
:103F300067E7120048E4939000861269E1ECF0AE66
:103F400059AF5A9067E7120048E4939000861269CF
:103F5000E1E0FC9067E9120048ECFCE493FDECD34F
:103F60009D40199067E9120048E493FC9067E712BE
:103F70000048E4939000861269E1ECF0AE59AF5A24
:103F8000742D6F4E7006755A33755900AE59AF5A7D
:103F900074022FFF50010E8E598F5A785A740126E1
:103FA000F6500418E436F64003023EE522E50C9094
:103FB000628AF828287302404A75E700A22FB340AE
:103FC00008E5B54408F5B58006E5B554F7F5B575CF
:103FD000E710807675E700A22FB34008E5B54440AE
:103FE000F5B58006E5B554BFF5B575E710805B758E
:103FF000E700A22FB34008E5B54480F5B58006E59B
:10400000B5547FF5B575E7108040A22F9287803AAE
:10401000A22F9290803475E700A22FB34008E5B537
:104020004410F5B58006E5B554EFF5B575E7108099
:104030001975E700A22FB34008E5B54420F5B58017
:0A40400006E5B554DFF5B575E7108D
:10628A00023FB6023FB9023FD4023FEF02400A0280
:08629A004010024016024031E1
:10404A002285F97285FA737E017F00E5731269B0E1
:10405A00E5722FFF50010E8E598F5AAC5BAD5CEFA3
:10406A002DFDEE3CFC8C5B8D5C1234B01234BB121D
:10407A0034C61234D19000CEE0B4032C75A7108553
:10408A00F97285FA737E017F00E5731269B0E572F1
:10409A002FFF50010E8E598F5A1234DC1234E71258
:1040AA0034F212350175A7002275A71085F97285B9
:1040BA00FA737E017F00E5731269B0E5722FFF5033
:1040CA00010E8E598F5A7E017F7690010BE012699C
:1040DA00B0AC59AD5AED2FFFEC3EFE8E5B8F5CE51E
:1040EA005CF5FDE55BF5FE900078E4F075A70074D9
:1040FA001290005DF02285F97285FA737E017F00C5
:10410A00E5731269B0E5722FFF50010E8E598F5A6E
:10411A00900019E0FCA3E0FDEF2DFDEE3CFC8C5B6A
:10412A008D5CE55CF5FDE55BF5FE220563229000FA
:10413A00CEE0640360079000ECE0B4021EA2D8B39C
:10414A004002C293A2D9B34002C294A2DAB3400297
:10415A00C291A2DBB34002C2928044A2D8B3400A01
:10416A00C2939000ECE06002C287A2D9B3400AC2AF
:10417A00949000ECE06002C290A2DAB3400EC291C1
:10418A009000ECE06006E5B554EFF5B5A2DBB3406C
:10419A000EC2929000ECE06006E5B554DFF5B5A2D8
:1041AA00DCB34030A2965006741990005DF0A295D7
:1041BA005006741990005DF0A2A050067419900080
:1041CA005DF0A2975006741990005DF0C296C295F0
:1041DA00C2A0C29775D8402285A77175A710900012
:1041EA00CEE0640360079000ECE0B40224A2D8B3E6
:1041FA004002C287A2D9B34002C290A2DAB34006F3
:10420A00E5B554EFF5B5A2DBB34006E5B554DFF5E5
:10421A00B5A2DCB340089000DAE0900078F075D8D7
:10422A00408571A72290F800E4936406600280FE3C
:10423A0075B50075840175A70075FF8075EF069046
:10424A000059E4F075C91075A70F75A1C775A700C5
:10425A0075D90075CE0C75A70F75F1FE75F2FF754D
:10426A00F30775F47875A4BA75A5FF75A60775AE38
:10427A000075AFFF75D48175D5FF75D6FF75D7FF69
:10428A0075A70075A20175A14775F80975D800755B
:10429A00D90475DA0975DB0975DC0975DD0975DE7E
:1042AA000975D84075A71075D80075D90475DA094B
:1042BA0075DB0975DC0975DD0975DE0975D8407588
:1042CA00A70075E60875E71075BC0175BE0475BDD3
:1042DA006C75BE0775BDA075BE0875BD0175BC00BD
:1042EA0075BB1875BC2075BA0875E88075D1137549
:1042FA00A70F75E10575E20075C740123C6D759709
:10430A0000759780740A1269907597C0E5975420D2
:10431A00700280F8758F0275A700D2AF7598007584
:10432A00A90C75A70F75AB4375ADFB75AC1E75A7C8
:10433A001075C91875CA0075CB0075C80475A70031
:10434A00758912758E04758C00758A00C2A9D28C83
:10435A00758D00758B00D2ABD28E75B62075D94497
:10436A00C299C22574C8F5097508001200F875A724
:10437A000FE5FB900067F0E5FA900068F0E5F99028
:10438A000069F075A70090F800E493F52612021769
:10439A00900899E0D394035007900899E0B4010675
:1043AA007400900899F074019000CFF0900899E099
:1043BA009062A2F8282873802A802875A70F75F3BF
:1043CA000F75A700A2A3400674029000CFF08013D5
:1043DA0075A70F75F31775A700A2A440067402907B
:0343EA0000CFF011
:0C62A2000243C10243C30243C50243DAB9
:1043ED009000CFE0B4022AC2241205B674029000E8
:1043FD00CFF0900899E09062AEF828287380108075
:0F440D000E74009000DEF0800674009000EBF05B
:0C62AE0002440A02440C02440E02441692
:10441C008028D2241204D574019000CFF090089912
:10442C00E09062BAF82828738010800E7400900017
:0A443C00DEF0800674009000EBF043
:0C62BA00024434024436024438024440DE
:104446001233109000D9E07006740A9000D9F090EB
:1044560000BAE0700674E39000BAF09000C0E00481
:1044660090007BF012359790F807E49390006EF079
:1044760090006EE0440A90006EF090006EE054FEEC
:1044860090006EF0740690005FF07401900060F08A
:1044960090F802E493900061F07403900062F07467
:1044A60005900063F0742B900064F074069000652C
:1044B600F0900061E0B405067405900065F074069E
:1044C600900066F090F804E49390006AF07400900F
:1044D600006BF090F805E49390006CF090F806E419
:1044E6009390006DF074FF90006FF0123D529000B3
:1044F60061E0B40505123EDF8003123E119000F51F
:10450600E0900074F09000ACE0900075F09000AD83
:10451600E0900076F0A2B6B39204A2B3B39205A2DD
:10452600A4B3921EA2A3B3921F900070E4F0756E1E
:1045360000743A900786F074FD900787F09000713A
:10454600E4F0756D0190005DE4F09000D0E0B401F8
:1045560006741A90005DF0C21D756200C209D20A87
:10456600C202757000C22012009E755E00756A0058
:10457600756000756432756500756600756700754F
:10458600680075690090001FE4F0A3F0756B00D217
:10459600B2D2A4D2B0D2B1D2A3D2A7D2A6D2A5D239
:1045A600B7900092E0D394FA400674FA900092F025
:1045B6007E017F00900076E01269B0900075E02FD2
:1045C600FF50010E900029EEF0A3EFF0EFD394FF19
:1045D600EE940F4007900029E4F0A3F0900074E0F9
:1045E600700674FF900074F09000D0E07005756C52
:1045F600028003756C039000D1E0D39401400674E9
:10460600009000D1F09000D7E0C3940A5006740AD7
:104616009000D7F09000E1E0700674019000E1F0A0
:104626009000E1E0B4FF0674FE9000E1F09000E82F
:10463600E0D394FE400674FE9000E8F090010EE090
:10464600D394024006740190010EF0900124E0D349
:10465600940140067401900124F074019000EEF07C
:1046660074019000EFF074009000F6F07419900158
:1046760013F0741A900114F0742A900115F0740066
:10468600900116F074299006CCF0D29C9000C1E0FF
:10469600D39404400674049000C1F09000F3E0D374
:1046A6009404400674049000F3F0E56FD394104030
:1046B60003756F109006CDE0D3940C4006740090FD
:1046C60006CDF09006D1E0D3940C40067400900617
:1046D600D1F09006D5E0D3940C400674009006D530
:1046E600F09006D9E0D3940C400674009006D9F0F9
:1046F6009006DDE0D3940C400674009006DDF09041
:1047060006E1E0D3940C400674009006E1F09006B2
:10471600E5E0D3940C400674009006E5F0D2EC7503
:10472600CF01A298B34005C298120697E54C6006E1
:10473600A299B3B340028005C299120B78E54D6485
:10474600016005E54DB4040280D5C28E7E107F005F
:10475600E5631269B0E58D75F010A4FDACF0EF2DA0
:10476600FDEE3CFCE58B75F01084FF7E00ED2FFF1F
:10477600EC3EFE8E538F54D28E9000B3E0600990CB
:1047860000B3E0C3943D4002805C9000211269BEF4
:10479600900021E0FEA3E0FF900023E0FCA3E0FDF3
:1047A600EFB50542EEB5043EB217A203B340197544
:1047B600E700A217B34008E5B54404F5B58006E561
:1047C600B554FBF5B575E710900023E0FEA3E0FFB6
:1047D600900025E0FCA3E0FDEF2DFDEE3CFC9000F3
:1047E60023ECF0A3EDF09000C0E060099000C0E07B
:1047F600C394034003024889122745A203B3500914
:10480600900070E0C3942B400280069000AAE0F569
:1048160044E54475F002A4FFAEF090088EEEF0A3D6
:10482600EFF0900097E0C395604007E55EC3955FA3
:10483600500790088EE4F0A3F075E700AE2DAF2E7A
:1048460090088EE0FCA3E0FDEFD39DEE9C4015E5BD
:10485600B554F7F5B59000C0E0B40206E5B54402DC
:10486600F5B5801C900070E0C394415013E5B54443
:1048760008F5B59000C0E0B40206E5B554FDF5B5FF
:1048860075E7109000C0E0B4032A12286075E700AF
:10489600AE2DAF2E90088EE0FCA3E0FDEFD39DEE8B
:1048A6009C4008E5B54408F5B58006E5B554F7F52E
:1048B600B575E71090009BE06009A2B3300501B31F
:1048C600B340028028A2B3300501B34020A2B33022
:1048D6000701B3400B900081E004F0A207B39205F4
:1048E600A207B330B301B34004A2079205A2B630C3
:1048F6000401B35003024FE7A2B6300401B35003DC
:10490600024FE7A2B6300601B35003024E51756D51
:10491600009000B3E0B43D1975E700A206B3400865
:10492600E5B554FBF5B58006E5B54404F5B575E780
:1049360010055DA208B3B35013AE53AF54900010E8
:10494600E0FCA3E0FDEDC39FEC9E4003024AFEE5BA
:104956006CB40375A226B34022E55DB41203756CF0
:1049660001E55DC39412500690005D7401F0E55DAB
:10497600D394124006740290005DF0900081E064CA
:10498600016007900081E0B40405755D01801A900E
:104996000081E064026007900081E0B40305755D64
:1049A600138006740590005DF0900081E0B401026A
:1049B600D21A900081E0B40402C21AD22690008175
:1049C600E0B40102D21A024A70E56CB40206756CB4
:1049D60001755D12E55D64126005E55DB4244290E3
:1049E6000081E064016007900081E0B40405755D14
:1049F60001801A900081E064026007900081E0B4B3
:104A06000305755D138006740590005DF0900081C6
:104A1600E0B40102D21A900081E0B40402C21A8006
:104A26004990005DE07034E55DC394125006900035
:104A36005D7401F0E55DD394124006740290005D4A
:104A4600F0E55DC394125002D21DE55DD394124089
:104A560002D21DC296C295C2A0C2979000D0E0B401
:104A66000105123C6D8003755D01AE55AF56AC5322
:104A7600AD54EF2DFDEE3CFC7403FF1269A08C557E
:104A86008D569000B3E060099000B3E0C3943D40BA
:104A9600028049900021E0FEA3E0FF9000B3E08E83
:104AA600048F05FF1269A074018C068D0712003968
:104AB600900025EEF0A3EFF0900025E0F8A3E0903B
:104AC6000023C8F0A3C8F0900021E4F0A3F0C217B9
:104AD60075E700E5B554FBF5B575E710A2A4B3403C
:104AE60002C21EA2A3B34002C21FA21DB34002C24D
:104AF6001D900081E4F0803AAE55AF56AC53AD54EC
:104B0600EF2DFDEE3CFC74018C068D071200398EEC
:104B1600558F56E56CC39402500DAC53AD54748852
:104B2600C39D74139C40028009123C6D740690006C
:104B36005DF0E55DB41212740390005DF0D21D9035
:104B460000D0E0B40103123C6DAE57AF58AC53AD84
:104B560054EF2DFDEE3CFC8C578D58AE53AF54EF01
:104B6600D39DEE9C4011900017E0FAA3E0FBEBC347
:104B760094E8EA9403400280069000171269BE90FA
:104B86000014E0FEA3E0FFAC53AD54EF2DFDEE3C68
:104B9600FC900014ECF0A3EDF09000D0E0B4011D01
:104BA600AE53AF5474051269B074038E048F05FFBB
:104BB6001269A0900010ECF0A3EDF08016AE53AF92
:104BC6005474031269B07401120039900010EEF0AB
:104BD600A3EFF0C28E758D00758B0075630075545A
:104BE60001755300D28EE55D240875F00984AFF097
:104BF6007E00EF4E6003024C81E56C6013AE55AF4C
:104C06005674091269B0900012EEF0A3EFF0800F0F
:104C1600900014E0F8A3E0900012C8F0A3C8F0904A
:104C26000012E0FEA3E0FFEF4E600B7C7D7D741268
:104C3600689E8E518F52900014E4F0A3F0AE51AFEF
:104C4600527428BE00039F5010E5622FFF50010EDC
:104C560074011200398E518F528552629000D7E04E
:104C6600A851B8000DD395524008E55290005CF06B
:104C760080099000D7E01490005CF09000CEE0B47C
:104C86000308900051E0655D6002800EA21A301B99
:104C960001B34004D21C8002C21CE55D640B6005B2
:104CA600E55DB41D099000C0E06003122411900078
:104CB6005AE0655D600790005BE0B55D03756E00C8
:104CC600A209B35006A208B3B34003024D7990007F
:104CD6008CE0B4017390010EE0B40214120D199029
:104CE6000079E075F0BEA4FFAEF08E5B8F5C805657
:104CF600E56675F00A84FF7E00900586120048E09E
:104D0600F55A755900AE59AF5A9000B1E01269B024
:104D160074648E048F05FF1269A08C5B8D5CE55C64
:104D2600900016F0AE59AF5A90008AE01269B0743E
:104D3600648E048F05FF1269A074BE8C068D07125F
:104D460069B08E5B8F5C801790008AE075F0BEA418
:104D5600FFAEF08E5B8F5C9000B1E0900016F0E540
:104D660060C394CC5006E55C455B7002800312403C
:104D76004BD209E56CB40106E55D640B6002800C5C
:104D8600756F0190005E7401F0756C00E56C600350
:104D9600024E4C9000D3E0600D900078E0A851B828
:104DA60000069552400280489000D3E0B402279056
:104DB600004DE0655D601790004EE0655D600F9008
:104DC600004FE0655D6007900050E0B55D03756FCC
:104DD60003756B00800CC200756B0090001FE4F039
:104DE600A3F0900078E06006740990005DF08056AC
:104DF60090004DE0655D601790004EE0655D600FC8
:104E060090004FE0655D6007900050E0B55D377536
:104E16006F0190004DE0B55D0690005E7401F09064
:104E2600004EE0B55D06740290005EF090004FE023
:104E3600B55D06740390005EF0900050E0B55D0627
:104E4600740490005EF0A206B39204A206B330B6D4
:104E560001B35003024FE7756D019000B3E0B43D16
:104E66001975E700A206B34008E5B54404F5B58018
:104E760006E5B554FBF5B575E710A225400575FFA7
:104E8600A0D22575E700E5B54401F5B575E71074C0
:104E96002B900070F0A2069204E55DD3944A40146C
:104EA600D208E55DD3946E400B740490005DF0D299
:104EB6001D755D469000DBE0B40107E569C39414F7
:104EC60040028009123C6D741390005DF075E70096
:104ED600900109E0A851B80005D39552500D9001F4
:104EE60008E0A851B80004955250028008E5B54480
:104EF60002F5B5801790010AE0D395604008E5B544
:104F06004402F5B58006E5B554FDF5B575E710E53F
:104F160069C394415009740E90005DF0123C6D9087
:104F26000065E0FE900061E0C39E4009900061E0EC
:104F3600D39408400974FB90005DF0123C6D90001C
:104F46006AE0601590006AE0FE900064E06E600919
:104F560074FE90005DF0123C6D900899E06006903A
:104F6600010BE06002807A74019000CFF0900899FE
:104F7600E09062C6F828287380188016A2A340061F
:104F860074029000CFF0800AA2A44006740290003A
:024F9600CFF05A
:0C62C600024F7E024F80024F82024F8E7A
:104F98009000CFE0B40105A224B340028019D224C6
:104FA800123C6D1204D574019000CFF0123310D268
:104FB80020741B90005DF09000CFE0B40206A2249C
:104FC800B3B340028019C224123C6D1205B67402B4
:104FD8009000CFF0123310D220741B90005DF0A225
:104FE8001DB34008C296C295C2A0C29790010BE0BB
:104FF800600CAE51AF527414BE00059F400280375A
:10500800900093E09062D2F8282873802A8028A222
:10501800A3B35005A21FB3400280051240B3D21FAC
:105028008015A2A4B35005A21EB340028005124009
:07503800B3D21E80028000CC
:1062D20002501302501502501702502A02503D027A
:0262E200503F2B
:10503F00A20BB3B35008900051E0655D60030251BD
:10504F0086A201B35006A200B3B3400302517E9073
:10505F0000CEE0B403028003025145A21CB34058B6
:10506F0012345390011FE0601F90001DE0FEA3E07B
:10507F00FF900117E01269B074C88E048F05FF12FC
:10508F0069A08C5B8D5C800A90001DE0F55BA3E04E
:10509F00F55CAE5BAF5C745E1269B074058E048F05
:1050AF0005FF1269A0AE59AF5AED2FFFEC3EFE8EF1
:1050BF005B8F5C1234B0805C12348090011FE0D3A0
:1050CF009404401F90001DE0FEA3E0FF90011BE041
:1050DF001269B074C88E048F05FF1269A08C5B8DA6
:1050EF005C800A90001DE0F55BA3E0F55CAE5BAF62
:1050FF005C745E1269B074058E048F05FF1269A08F
:10510F00AE59AF5AED2FFFEC3EFE8E5B8F5C123423
:10511F00DC75A7009000ECE0B4011975E700A2025E
:10512F00B34008E5B54480F5B58006E5B5547FF585
:10513F00B575E71080399000ECE0C39402500F1260
:10514F0034531234B0A202B34002D28780211234FA
:10515F00531234B0123480AE59AF5AAC2BAD2CEF82
:10516F002DFDEE3CFC8C5B8D5C1234DC75A700C210
:10517F000BD20CD20DD20EA20CB3B350089000522A
:10518F00E0655D60030252D0A201B35006A200B3E6
:10519F00B340030252C89000CEE0B4030280030272
:1051AF00528FA21CB3405B12345390011FE0D39473
:1051BF0001401F90001DE0FEA3E0FF900118E012D8
:1051CF0069B074C88E048F05FF1269A08C5B8D5C6B
:1051DF00800A90001DE0F55BA3E0F55CAE5BAF5C71
:1051EF00745E1269B074058E048F05FF1269A0AE4C
:1051FF0059AF5AED2FFFEC3EFE8E5B8F5C1234BB26
:10520F00805C12348090011FE0D39405401F900002
:10521F001DE0FEA3E0FF90011CE01269B074C88E80
:10522F00048F05FF1269A08C5B8D5C800A90001DB6
:10523F00E0F55BA3E0F55CAE5BAF5C745E1269B04A
:10524F0074058E048F05FF1269A0AE59AF5AED2F6A
:10525F00FFEC3EFE8E5B8F5C1234E775A70090006B
:10526F00ECE0B4011975E700A202B34008E5B544BC
:10527F0080F5B58006E5B5547FF5B575E710803933
:10528F009000ECE0C39402500F1234531234BBA2BF
:10529F0002B34002D29080211234531234BB123425
:1052AF0080AE59AF5AAC2BAD2CEF2DFDEE3CFC8CE4
:1052BF005B8D5C1234E775A700D20BC20CD20DD2F6
:1052CF000EA20DB3B35008900053E0655D6003026A
:1052DF00541EA201B35006A200B3B34003025416EA
:1052EF009000CEE0B4030280030253D9A21CB34056
:1052FF005B12345390011FE0D39403401F90001DA5
:10530F00E0FEA3E0FF900119E01269B074C88E04AB
:10531F008F05FF1269A08C5B8D5C800A90001DE0E9
:10532F00F55BA3E0F55CAE5BAF5C745E1269B074C5
:10533F00058E048F05FF1269A0AE59AF5AED2FFFEE
:10534F00EC3EFE8E5B8F5C1234C6805C1234809014
:10535F00011FE0D39406401F90001DE0FEA3E0FF65
:10536F0090011DE01269B074C88E048F05FF126999
:10537F00A08C5B8D5C800A90001DE0F55BA3E0F5CF
:10538F005CAE5BAF5C745E1269B074058E048F0502
:10539F00FF1269A0AE59AF5AED2FFFEC3EFE8E5BA8
:1053AF008F5C1234F275A7009000ECE0B401197510
:1053BF00E700A202B34008E5B54480F5B58006E5E5
:1053CF00B5547FF5B575E710803D9000ECE0C394C0
:1053DF000250131234531234C6A202B34006E5B57D
:1053EF004410F5B580211234531234C6123480AEF6
:1053FF0059AF5AAC2BAD2CEF2DFDEE3CFC8C5B8DD9
:10540F005C1234F275A700D20BD20CC20DD20EA2D1
:10541F000EB3B35008900054E0655D600302556C05
:10542F00A201B35006A200B3B3400302556490002B
:10543F00CEE0B403028003025527A21CB3405B12D7
:10544F00345390011FE0D39403401F90001DE0FEE2
:10545F00A3E0FF90011AE01269B074C88E048F05A3
:10546F00FF1269A08C5B8D5C800A90001DE0F55BDC
:10547F00A3E0F55CAE5BAF5C745E1269B074058E31
:10548F00048F05FF1269A0AE59AF5AED2FFFEC3E06
:10549F00FE8E5B8F5C1234D1805C12348090011FC2
:1054AF00E0D39407401F90001DE0FEA3E0FF9001A2
:1054BF001EE01269B074C88E048F05FF1269A08CAC
:1054CF005B8D5C800A90001DE0F55BA3E0F55CAEA0
:1054DF005BAF5C745E1269B074058E048F05FF12AA
:1054EF0069A0AE59AF5AED2FFFEC3EFE8E5B8F5C7D
:1054FF0012350175A7009000ECE0B4011975E700B3
:10550F00A202B34008E5B54480F5B58006E5B55471
:10551F007FF5B575E710803D9000ECE0C394025025
:10552F00131234531234D1A202B34006E5B544200E
:10553F00F5B580211234531234D1123480AE59AFE5
:10554F005AAC2BAD2CEF2DFDEE3CFC8C5B8D5C1221
:10555F00350175A700D20BD20CD20DC20EE56F909C
:0D556F0062E4F8282873025A429000F3E02D
:0662E40002557502557819
:10557C00906323F8282873121DB38012121DB38078
:0E558C000D121E3D8008121EE98003121EE95A
:0F63230002558302558802558D025592025597F7
:10559A00756F02025A4212201512212C12244690CB
:1055AA000886E0FEA3E0FF740A1269B0900012E0D8
:1055BA00FCA3E0FD74098F02FF1269A08D078C031A
:1055CA008E048A058B0612689E90088AEEF0A3EF75
:1055DA00F074F0BE00039F500B74F090088AF8E450
:1055EA00F0E8A3F0E535700375350190088AE0FE0E
:1055FA00A3E0FFE5352FFF50010E90088AEEF0A3D5
:09560A00EFF0756F0390005EE003
:0362EA000255A0BA
:10561300906332F82828738022A22E4003756F0A04
:105623008019A22E4003756F0B8010A22E400375C4
:0B5633006F0C8007A22E4003756F0D66
:0F63320002561A02561C02562502562E025637E4
:10563E00025A429006CDE060077401F50812256DFE
:10564E0090010CE0B4011490010DE0A851B80004D3
:10565E0095525007E55EC3955F4002800974159020
:10566E00005DF00256F59000C1E0D39402403F90E9
:10567E000095E02403A851B80004955250099000FB
:10568E0097E0D3956050028008D201740890005DB7
:10569E00F0900095E0A851B80005D39552500B90AC
:1056AE000097E02403C395605002C2018039900038
:1056BE0095E02403A851B8000495525007E55EC347
:1056CE00955F40028008D201740890005DF0900052
:1056DE0095E0A851B80005D395525009E55F240F07
:1056EE00C3955E5002C2019000DBE07007E569C30E
:1056FE00941440028002D2019000D0E0B40102D294
:10570E0001A2014005756F04800A756F1090001F8D
:0B571E00E4F0A3F0025A429000C1E04A
:0662ED0002564102572594
:10572900906341F8282873120E038012120E038029
:0E5739000D120FB1800812106380031210636E
:0F63410002573002573502573A02573F0257446E
:105747009006D1E060077402F50812256D756F05A4
:10575700025A421211A3756F069006D5E0600774CE
:1057670003F50812256D9006D9E060077404F50863
:1057770012256D025A42900016E06006A203B3B3E9
:105787004002801D900016E02528FFAE2750010E2D
:105797008E278F28E55DD394095006900016E014F4
:1057A700F01213E9756F079006DDE060077405F5E1
:1057B7000812256D9006E1E060077406F5081225CA
:1057C7006D025A4290010EE0B40203120D911218B5
:1057D70019756F089006E5E060077407F50812254C
:1057E7006D025A42121BD5A20BB35005A20CB3404F
:1057F700028008D20BD20CD20DD20E756F10025A4E
:1058070042025A4290003FE0C394465008C2967441
:105817004690003FF0900055E0B4011DE535240A9D
:10582700F53590088AE0FEA3E0FF740A2FFF5001C8
:105837000E90088AEEF0A3EFF085355A755900905F
:10584700004DE0F572123510E55C90003FF09000D6
:1058570008E559F0A3E55AF0E572900040F0C21050
:1058670090088AE0F559A3E0F55A90004DE0F572EB
:10587700123510E55C90003DF0900000E559F0A36B
:10588700E55AF0E57290003EF0C20F756F03025AB9
:1058970042900043E0C394465008C2957446900076
:1058A70043F0900056E0B4011DE535240AF5359024
:1058B700088AE0FEA3E0FF740A2FFF50010E90084C
:1058C7008AEEF0A3EFF085355A75590090004EE047
:1058D700F572123510E55C900043F090000AE55927
:1058E700F0A3E55AF0E572900044F0C21290088ADE
:1058F700E0F559A3E0F55A90004EE0F57212351025
:10590700E55C900041F0900002E559F0A3E55AF0FC
:10591700E572900042F0C211756F03025A4290007F
:1059270047E0C394465008C2A07446900047F090E1
:105937000057E0B4011DE535240AF53590088AE0E3
:10594700FEA3E0FF740A2FFF50010E90088AEEF0C5
:10595700A3EFF085355A75590090004FE0F57212A4
:105967003510E55C900047F090000CE559F0A3E591
:105977005AF0E572900048F0C21490088AE0F55991
:10598700A3E0F55A90004FE0F572123510E55C90F0
:105997000045F0900004E559F0A3E55AF0E5729050
:1059A7000046F0C213756F03025A4290004BE0C3E2
:1059B70094465008C297744690004BF0900058E008
:1059C700B4011DE535240AF53590088AE0FEA3E009
:1059D700FF740A2FFF50010E90088AEEF0A3EFF034
:1059E70085355A755900900050E0F572123510E56B
:1059F7005C90004BF090000EE559F0A3E55AF0E5F6
:105A07007290004CF0C21690088AE0F559A3E0F5B1
:105A17005A900050E0F572123510E55C900049F09D
:105A2700900006E559F0A3E55AF0E57290004AF0B8
:0B5A3700C215756F0380048002800020
:1062F30002575A02577D0257CB0257EB0258080246
:10630300580B0258980259250259B2025A3E025AB2
:0463130040025A42A8
:105A420090003DE0B55D73A20F404F900000E0FE74
:105A5200A3E0FFEF4E6021AE55AF56900000E0FC90
:105A6200A3E0FD120003740A8E048F05FF1269A0E1
:105A7200900000ECF0A3EDF090003EE0601A900080
:105A820000E0FEA3E0FFAC55AD56EF2DFDEE3CFC71
:105A9200900000ECF0A3EDF0D20FAE53AF549000A3
:105AA20000E0FCA3E0FDEFC39DEE9C400D1241001F
:105AB200D296C20F74C890003DF0A20FB3B3500744
:105AC20090003DE0B55D02800D124100D29674C88F
:105AD20090003DF0C20F90003FE0B55D70A2104013
:105AE2004F900008E0FEA3E0FFEF4E6021AE55AFFD
:105AF20056900008E0FCA3E0FD120003740A8E0435
:105B02008F05FF1269A0900008ECF0A3EDF0900061
:105B120040E0601A900008E0FEA3E0FFAC55AD56ED
:105B2200EF2DFDEE3CFC900008ECF0A3EDF0D2105E
:105B3200AE53AF54900008E0FCA3E0FDEFC39DEE2E
:105B42009C400AC296744690003FF0C210A210B365
:105B5200B3500790003FE0B55D02800AC2967446DA
:105B620090003FF0C210900041E0B55D73A2114079
:105B72004F900002E0FEA3E0FFEF4E6021AE55AF72
:105B820056900002E0FCA3E0FD120003740A8E04AA
:105B92008F05FF1269A0900002ECF0A3EDF09000D7
:105BA20042E0601A900002E0FEA3E0FFAC55AD5661
:105BB200EF2DFDEE3CFC900002ECF0A3EDF0D211D3
:105BC200AE53AF54900002E0FCA3E0FDEFC39DEEA4
:105BD2009C400D124100D295C21174C8900041F050
:105BE200A211B3B35007900041E0B55D02800D12DF
:105BF2004100D29574C8900041F0C211900043E078
:105C0200B55D70A212404F90000AE0FEA3E0FFEFE4
:105C12004E6021AE55AF5690000AE0FCA3E0FD12A3
:105C22000003740A8E048F05FF1269A090000AEC2B
:105C3200F0A3EDF0900044E0601A90000AE0FEA3A9
:105C4200E0FFAC55AD56EF2DFDEE3CFC90000AECAA
:105C5200F0A3EDF0D212AE53AF5490000AE0FCA3D1
:105C6200E0FDEFC39DEE9C400AC29574469000434E
:105C7200F0C212A212B3B35007900043E0B55D0226
:105C8200800AC2957446900043F0C212900045E02B
:105C9200B55D73A213404F900004E0FEA3E0FFEF56
:105CA2004E6021AE55AF56900004E0FCA3E0FD1219
:105CB2000003740A8E048F05FF1269A0900004ECA1
:105CC200F0A3EDF0900046E0601A900004E0FEA31D
:105CD200E0FFAC55AD56EF2DFDEE3CFC900004EC20
:105CE200F0A3EDF0D213AE53AF54900004E0FCA346
:105CF200E0FDEFC39DEE9C400D124100D2A0C21305
:105D020074C8900045F0A213B3B35007900045E069
:105D1200B55D02800D124100D2A074C8900045F01A
:105D2200C213900047E0B55D70A214404F90000C82
:105D3200E0FEA3E0FFEF4E6021AE55AF5690000C9F
:105D4200E0FCA3E0FD120003740A8E048F05FF122B
:105D520069A090000CECF0A3EDF0900048E0601A0E
:105D620090000CE0FEA3E0FFAC55AD56EF2DFDEE2A
:105D72003CFC90000CECF0A3EDF0D214AE53AF5407
:105D820090000CE0FCA3E0FDEFC39DEE9C400AC234
:105D9200A07446900047F0C214A214B3B350079007
:105DA2000047E0B55D02800AC2A07446900047F049
:105DB200C214900049E0B55D73A215404F900006F1
:105DC200E0FEA3E0FFEF4E6021AE55AF5690000615
:105DD200E0FCA3E0FD120003740A8E048F05FF129B
:105DE20069A0900006ECF0A3EDF090004AE0601A82
:105DF200900006E0FEA3E0FFAC55AD56EF2DFDEEA0
:105E02003CFC900006ECF0A3EDF0D215AE53AF547B
:105E1200900006E0FCA3E0FDEFC39DEE9C400D1256
:105E22004100D297C21574C8900049F0A215B3B3CD
:105E32005007900049E0B55D02800D124100D297F3
:105E420074C8900049F0C21590004BE0B55D70A295
:105E520016404F90000EE0FEA3E0FFEF4E6021AE31
:105E620055AF5690000EE0FCA3E0FD120003740A49
:105E72008E048F05FF1269A090000EECF0A3EDF0E6
:105E820090004CE0601A90000EE0FEA3E0FFAC55DB
:105E9200AD56EF2DFDEE3CFC90000EECF0A3EDF0C4
:105EA200D216AE53AF5490000EE0FCA3E0FDEFC358
:105EB2009DEE9C400AC297744690004BF0C216A217
:105EC20016B3B3500790004BE0B55D02800AC2974B
:105ED200744690004BF0C2169000DEE0B4020280DD
:105EE2000302600E900072E0D395655064900072D8
:105EF200E0F4042565FE9000E1E08E00F5F0E88410
:105F0200FF7E008F72EFC39410500CEF8572F0A4E5
:105F1200FDACF08D7280037572FF900072E0D39534
:105F220072400B900072E0C39572F5708003757039
:105F3200009000FCE0D3957040069000FCE0F57004
:105F42009000FDE0C3957050069000FDE0F5708072
:105F520071900072E0C39565FE9000E1E08E00F55D
:105F6200F0E884FF7E008F72EFC39410500CEF852F
:105F720072F0A4FDACF08D7280037572FF85725AC7
:105F8200755900900072E0255AFFAE5950010E8EED
:105F9200598F5A74FFBE0009D39F4005855A7080FD
:105FA200037570FF9000FCE0D3957040069000FCF2
:105FB200E0F5709000FDE0C3957050069000FDE0A2
:105FC200F570A203B3B3500D900073E0FE9000E9A8
:105FD200E0D39E50028014740790005DF075E700D4
:105FE200E5B554BFF5B575E710802175A71075E7C3
:105FF20000E5CDC395704008E5B554BFF5B5800600
:10600200E5B54440F5B575E71075A700900103E0CA
:10601200A851B80005D395525016900102E0A8513C
:10602200B8000D95524009900104E0D395604002FA
:10603200802175A710A203B3B35007E5CDC394BF67
:1060420040028004D2A28002C2A2A2A292A175A79B
:1060520000801F75A710A203B3B35007E5CDC39408
:106062004040028004D2A28002C2A2A2A292A175E2
:10607200A700E56EC39409500AA2EDB34005C2ED34
:10608200122A07AE53AF547410C39F74279E400C5C
:10609200900071E0C3945A4003026287A208B340A1
:1060A20009123C6D740690005DF0A20AB3500EE531
:1060B20060D394334007E560C394CC4002804A9099
:1060C200010EE0B40214120D19900079E075F0503F
:1060D200A4FFAEF08E5B8F5C800F90008AE075F0BB
:1060E20050A4FFAEF08E5B8F5CE55C455B601AA24C
:1060F20025400575FFA0D225E5B54401F5B5742B01
:10610200900070F012404BD20A900071E0D39401DB
:106112004007E560C3941A40028002C20A9006CD8D
:10612200E060077401F50812256D9006D1E0600762
:106132007402F50812256D9006D5E060077403F528
:106142000812256D9006D9E060077404F50812253F
:106152006D9006DDE060077405F50812256D900666
:10616200E1E060077406F50812256D9006E5E0602F
:10617200077407F50812256D900071E0C3945A5018
:1061820026E56EB40909900071E004F0756E009086
:106192000071E0B45A0FA225400575FFA0D225E593
:1061A200B54401F5B5803BE56EB40903756E007523
:1061B2005400755300758D00758B00756300900057
:1061C20070E0C394415008900070E004F0800674BF
:1061D20041900070F0900070E0B44106E5B554FEC5
:1061E200F5B5900071E0D394014007E569C394418D
:1061F20040028009740E90005DF0123C6D90089987
:10620200E0600690010BE06002807A74019000CF9A
:10621200F0900899E0906317F82828738018801688
:10622200A2A3400674029000CFF0800AA2A4400606
:0662320074029000CFF0A1
:0C63170002621E02622002622202622E5C
:106238009000CFE0B40105A224B340028019D22413
:10624800123C6D1204D574019000CFF0123310D2B5
:1062580020741B90005DF09000CFE0B40206A224E9
:10626800B3B340028019C224123C6D1205B6740201
:106278009000CFF0123310D220741B90005DF00212
:026288004725A8
:106350000000010001400160018001A001C001E0D6
:1063600002000300039603B603D603F404000500FD
:106370000512052405360548055A056C057E05906D
:1063800005A805C005DE0600061406280646066EAA
:1063900006AE05CF00FF013F015F017F019F01BFF6
:1063A00001DF01FF02FF039503B503D503F303FFEC
:1063B00004FF05110523053505470559056B057DC6
:1063C000058F05A705BF05CE05F10613062706456F
:1063D000066D06AD06ED05DD0FAA0FA50F9F0F9AFE
:1063E0000F940F8D0F870F800F780F710F680F605C
:1063F0000F570F4E0F450F3B0F300F250F1A0F0E83
:106400000F020EF50EE80EDB0ECC0EBE0EAE0E9F8A
:106410000E8E0E7D0E6C0E5A0E470E340E200E0C94
:106420000DF70DE20DCB0DB50D9D0D850D6D0D54C8
:106430000D3A0D200D050CE90CCE0CB10C940C7628
:106440000C580C3A0C1B0BFB0BDB0BBB0B9A0B79A0
:106450000B570B350B130AF10ACE0AAB0A870A64F5
:106460000A400A1C09F809D409B0098C09670943D4
:10647000091F08FB08D608B2088E086A08460823D8
:1064800007FF07DC07B9079607730751072F070DAA
:1064900006EC06CA06AA068906690649062A060AFD
:1064A00005EC05CD05B0059205750558053C0520A0
:1064B000050504EA04CF04B5049C04820469045170
:1064C00004390422040B03F403DE03C803B2039D62
:1064D000038903750361034D033B0328031603047B
:1064E00002F202E102D102C002B002A002910282D5
:1064F0000273026502570249023C022F0222021671
:10650000020901FD01F201E601DB01D001C601BB78
:1065100001B101A7019D0194018B018201790170F4
:1065200001680160015801500148014101390132FF
:10653000012B0125011E01180111010B010500FFAE
:1065400000FA0FA60FA00F990F920F8B0F840F7CEC
:106550000F740F6B0F620F580F4E0F430F380F2C35
:106560000F1F0F120F050EF70EE80ED80EC80EB74C
:106570000EA50E930E800E6C0E580E420E2C0E15AC
:106580000DFD0DE40DCB0DB10D950D790D5D0D3F9C
:106590000D200D010CE10CC00C9E0C7C0C590C352F
:1065A0000C100BEA0BC40B9E0B760B4F0B260AFD4F
:1065B0000AD40AAA0A800A550A2A09FF09D409A896
:1065C000097C0950092508F908CD08A10875084A71
:1065D000081E07F307C8079D07730749072006F73A
:1065E00006CE06A6067E06570630060A05E405BF57
:1065F000059B057705540532051004EF04CE04AE63
:10660000048F047104530435041903FD03E203C726
:1066100003AD0394037B0363034B0334031E03089E
:1066200002F302DE02CA02B602A30291027F026DE9
:10663000025C024C023C022C021D020E020001F21E
:1066400001E401D701CA01BE01B101A6019A018F7F
:106650000185017A01700166015D0153014A014122
:10666000013901310129012101190112010B010434
:1066700000FD00F700F000EA00E400DE00D900D3DE
:1066800000CE00C900C400BF00BA00B500B100AD23
:1066900000A800A400A0009C009900950091008E25
:0C66A000008A008700840081007E007BDF
:10009E00754600900890E4F0A3F0753000752F00BF
:1000AE00754C00754D00C229D22B900899E0600264
:1000BE00D22074FE900892F8E4F0E8A3F074FE905B
:1000CE000896F8E4F0E8A3F074FE900894F8E4F0D3
:1000DE00E8A3F0745A9008B8F0745A9008B9F0D2A8
:1000EE002CC227C22EC22DC22822750B00750A0003
:1000FE00AE0AAF0BAC08AD09EDC39FEC9E40167473
:10010E00FF12699075CF01780B740126F650041812
:10011E00E436F650DB22C2AF75D904758F0375B77E
:10012E00A575B7F190F800E4F0758F0175B7A57558
:10013E00B7F1E52690F800F075B7A575B7F190F810
:10014E0001E4F075B7A575B7F19008ACE090F80230
:10015E00F075B7A575B7F19008B0E090F803F0759B
:10016E00B7A575B7F19008ADE090F804F075B7A596
:10017E0075B7F19008AEE090F805F075B7A575B7B4
:10018E00F19008AFE090F806F075B7A575B7F1904D
:10019E0008B1E090F807F0758F0075D944D2AF2200
:1001AE00900059E0B4AB61C2AF75D90475B6227533
:1001BE00F522758F0375B7A575B7F1740090F6002B
:1001CE00F0758F01755A00755900AE59AF5A7413F8
:1001DE00BE00279F402475B7A575B7F190089812F9
:1001EE000048E0FC90F600120048ECF0785A7401DA
:1001FE0026F6500418E436F650D0758F0075F511BA
:10020E0075B62075D944D2AF22C2AF75F52275D915
:10021E0004755A00755900AE59AF5A7413BE0022B8
:10022E009F401F90F600120048E493FC900898122D
:10023E000048ECF0785A740126F6500418E436F6AD
:10024E0050D575D94475F511D2AF22900059E0B44E
:10025E00AA028003020396C2AF75D90475B6227541
:10026E00F522758F0375B7A575B7F1740090EE0082
:10027E00F075B7A575B7F1740090F000F075B7A5DD
:10028E0075B7F1740090F200F075B7A575B7F174FB
:10029E000090F400F0758F01755A00755900AE5933
:1002AE00AF5A74FFC39F74019E402475B7A575B7EE
:1002BE00F1900086120048E0FC90EE00120048EC2F
:1002CE00F0785A740126F6500418E436F650CF75BD
:1002DE005A00755900AE59AF5A74FFC39F74019EF0
:1002EE00402475B7A575B7F1900286120048E0FC60
:1002FE0090F000120048ECF0785A740126F6500483
:10030E0018E436F650CF755A00755900AE59AF5AEB
:10031E0074FFC39F74019E402475B7A575B7F19005
:10032E000486120048E0FC90F200120048ECF078CF
:10033E005A740126F6500418E436F650CF755A005A
:10034E00755900AE59AF5A74FFC39F74019E402475
:10035E0075B7A575B7F1900686120048E0FC90F4CB
:10036E0000120048ECF0785A740126F6500418E496
:10037E0036F650CF758F0075F51175B62075D944C8
:10038E00D2AF743A900786F022900059E0B4AA02D8
:10039E0080030204D4C2AF75D90475B62275F52256
:1003AE00758F0375B7A575B7F1740090E600F075FB
:1003BE00B7A575B7F1740090E800F075B7A575B7DD
:1003CE00F1740090EA00F075B7A575B7F17400905E
:1003DE00EC00F0758F01755A00755900AE59AF5A81
:1003EE0074FFC39F74019E402475B7A575B7F19035
:1003FE000086120048E0FC90E600120048ECF0780F
:10040E005A740126F6500418E436F650CF755A0089
:10041E00755900AE59AF5A74FFC39F74019E4024A4
:10042E0075B7A575B7F1900286120048E0FC90E80A
:10043E0000120048ECF0785A740126F6500418E4C5
:10044E0036F650CF755A00755900AE59AF5A74FF33
:10045E00C39F74019E402475B7A575B7F1900486AD
:10046E00120048E0FC90EA00120048ECF0785A7452
:10047E000126F6500418E436F650CF755A00755919
:10048E0000AE59AF5A74FFC39F74019E402475B7D6
:10049E00A575B7F1900686120048E0FC90EC0012AC
:1004AE000048ECF0785A740126F6500418E436F63B
:1004BE0050CF758F0075F51175B62075D944D2AF32
:1004CE00743A900786F022C2AF75D90475F522757D
:1004DE005A00755900AE59AF5A74FFC39F74019EEE
:1004EE00401F90EE00120048E493FC90008612002C
:1004FE0048ECF0785A740126F6500418E436F6509B
:10050E00D4755A00755900AE59AF5A74FFC39F7413
:10051E00019E401F90F000120048E493FC9002866A
:10052E00120048ECF0785A740126F6500418E4369E
:10053E00F650D4755A00755900AE59AF5A74FFC3B0
:10054E009F74019E401F90F200120048E493FC90AD
:10055E000486120048ECF0785A740126F6500418FE
:10056E00E436F650D4755A00755900AE59AF5A7428
:10057E00FFC39F74019E401F90F400120048E49345
:10058E00FC900686120048ECF0785A740126F6505C
:10059E000418E436F650D475F51175D944D2AF74FB
:1005AE003A900786F0C22A22C2AF75D90475F52299
:1005BE00755A00755900AE59AF5A74FFC39F740136
:1005CE009E401F90E600120048E493FC90008612B5
:1005DE000048ECF0785A740126F6500418E436F60A
:1005EE0050D4755A00755900AE59AF5A74FFC39F57
:1005FE0074019E401F90E800120048E493FC9002A4
:10060E0086120048ECF0785A740126F6500418E46D
:10061E0036F650D4755A00755900AE59AF5A74FF5C
:10062E00C39F74019E401F90EA00120048E493FCA1
:10063E00900486120048ECF0785A740126F65004A5
:10064E0018E436F650D4755A00755900AE59AF5AA3
:10065E0074FFC39F74019E401F90EC00120048E48B
:10066E0093FC900686120048ECF0785A740126F638
:10067E00500418E436F650D475F51175D944D2AF3E
:10068E00743A900786F0D22A22E54D64046006E59E
:10069E009964FF60028031A2294004D2298027E5A7
:1006AE004D600874E6254D90005DF0E54C600874D1
:1006BE00F0254C90005DF0E54DB4010280FE754DC5
:1006CE0000754C00C2298002C229E54D903280F897
:1006DE00282873754D00E599B4FF03754C01E59913
:1006EE00B4FE03754C02E599B4FD03754C03E59910
:1006FE00B4FC03754C04E599B4FA03754C05E59901
:10070E00B4FB06754D01123C6DE599B4F906754DB5
:10071E0004123C6DE599D394E54007E599C394F036
:10072E004002801685994E754D027E017F00E54E82
:10073E00C394E61269B08E318F32900890E4F0A324
:10074E00F0E599D394C44007E599C394E64002803E
:10075E002885994E754D0374E5C3954EF532753166
:10076E0000AE31AF3290635012697FE493F874019A
:10077E0093900890C8F0A3C8F0D299020B77900816
:10078E0098E0700AA221B35005A222B34002804223
:10079E00900890E0FEA3E0FF74FFBE00039F500997
:1007AE00EFC39446EE94064011900890E0FEA3E04D
:1007BE00FFEFD3946DEE94064013900890E0FEA3E5
:1007CE00E0FF900086120048E599F080038599734A
:1007DE008011900890E0FEA3E0FF90008612004882
:1007EE00E599F09008901269BE900890E0FEA3E0A3
:1007FE00FFEFB40106EEB407028003020970900702
:10080E0086E0B43C028003020970A221B35005A217
:10081E0022B340030208E7C29C900898E09001249E
:10082E00F0900899E0900093F090089AE09000B351
:10083E00F090089BE09000DCF090089CE09000881F
:10084E00F090089DE09000CEF090089EE09000ECB5
:10085E00F090089FE09000C0F09008A0E09000DEBD
:10086E00F09008A1E090010EF09008A2E0900172C5
:10087E00F09008A3E0900173F09008A4E09001744A
:10088E00F0123597900074E09000F5F0900075E04E
:10089E009000ACF0900076E09000ADF074AB90005C
:1008AE0059F01201AE74AA900059F0A22AB3400575
:1008BE001203978003120259900059E4F0900172CE
:1008CE00E0700C900173E07006900174E06002809D
:1008DE0004C2218002D221807EC29C900124E0902D
:1008EE000898F0900093E0900899F09000B3E09093
:1008FE00089AF09000DCE090089BF0900088E09061
:10090E00089CF09000CEE090089DF09000ECE090F6
:10091E00089EF09000C0E090089FF09000DEE090FE
:10092E0008A0F090010EE09008A1F074009008A2CB
:10093E00F074009008A3F074009008A4F074AB90CB
:10094E000059F01201AE74AA900059F01202591219
:10095E0003977599FB80FED29C754D00754C007502
:10096E0099FB020B77900890E0FEA3E0FFEF4E702C
:10097E0006859930752F00900890E0FEA3E0FF7475
:10098E00016F4E701BAC2FAD30AA31AB32ED2BFB8D
:10099E00EC3AFA8A068B07900086120048E599F029
:1009AE009008901269BE900890E0FEA3E0FF7402DA
:1009BE006F4E7021AC2FAD3074566D4C7006E54EF7
:1009CE0064E660028003123C6D123597854E997570
:1009DE004D00754C00020B77900890E0FEA3E0FFEF
:1009EE00900086120048E599F09008901269BE902A
:1009FE000890E0FEA3E0FFAC31AD328F028E038C87
:100A0E00068D0790639412697FE493F9740193FE47
:100A1E00EAD39EEB994009854E99754D00754C00B1
:100A2E00020B77900890E0FEA3E0FF900086120084
:100A3E0048E599F09008901269BE900890E0FEA3E8
:100A4E00E0FFEFB40006EEB401028003020B7790D4
:100A5E000069E0D394C7400B900069E0C394C8F5D9
:100A6E004F801A900069E0D39463400B900069E0C8
:100A7E00C39464F54F8006900069E0F54FE54F751D
:100A8E00F002A4FFAEF08F72EF9000861269E1EFD4
:100A9E00FCE0FDEC9000891269E1EDFCE0FDEC2D2F
:100AAE00B54F028003020B680FEF9000861269E1CA
:100ABE00E572FFE0FCEF90008A1269E1ECFFE0FCCA
:100ACE00EFC39CB54F028003020B68E5729000885D
:100ADE001269E1E572FFE0FCEF90008B1269E1EC28
:100AEE00FFE0FCEF2CB54F72E57290008C1269E1BD
:100AFE00E0C3954F9008ACF0E57290008D1269E15D
:100B0E00E0C3954F9008ADF0E5729000901269E148
:100B1E00E0C3954F9008AEF0E5729000911269E136
:100B2E00E0C3954F9008AFF0E5729000921269E124
:100B3E00E0C3954F9008B0F0E5729000931269E112
:100B4E00E0C3954F9008B1F01201247599F97464C1
:100B5E00F5097508001200F880FE7599FF7464F5AA
:090B6E00097508001200F880FE70
:0F3280000206E102078C0209730209E6020A3115
:100B770022E54C90328FF8282873020C5C9008907D
:100B8700E0FEA3E0FF90005F120048E0F5999008AF
:100B9700901269BE900890E0FEA3E0FF74116F4EBB
:100BA7007003754C00020C5C856D99020C5C900813
:100BB70090E0FEA3E0FF900086120048E0F599EF71
:100BC700B40107EEB40703754C009008901269BE94
:070BD700020C5C900891E0A4
:0F328F00020B81020B84020BAF020BB5020BDAAC
:100BDE009032E3F82828738552998067855E998054
:100BEE0062856099805D8564998058856699805389
:100BFE00856799804E85689980498569998044906A
:100C0E000020E0F599803CA22BB340077599FAC2FB
:100C1E002B8017A220B3400575990F800B90005DB5
:100C2E00E0F59990005DE4F0C2208017856A998006
:100C3E0012856599800D856B9980087599FC8003E6
:030C4E00754C00E2
:1032E300020BE5020BEA020BEF020BF4020BF902ED
:1032F3000BFE020C03020C08020C0D020C15020C4F
:0D3303003A020C3F020C44020C49020C4E31
:0B0C51009008901269BE80031233ED82
:03329E00020C59C6
:100C5C0022E536255AFFAE5950010E90008612003F
:100C6C0048E0F537E536255AFFAE5950010E0FBF57
:100C7C0000010E900086120048E0F538853E3AE5FA
:100C8C0037B538058537368041E538D39537401D63
:100C9C00E538C395378539F0A4FFAEF0E53A8E04FC
:100CAC008F05FF1269A0ED2537F536801DE537C39A
:100CBC0095388539F0A4FFAEF0E53A8E048F05FF28
:100CCC001269A0EDF4042537F53622E538D39537B3
:100CDC00401DE538C395378539F0A4FFAEF0E53AF1
:100CEC008E048F05FF1269A0ED2537F536801DE5C2
:100CFC0037C395388539F0A4FFAEF0E53A8E048FF2
:100D0C0005FF1269A0EDF4042537F5362290008C0E
:100D1C00E0B40170E56675F00A84FF7E008F36E55D
:100D2C006675F00A84ADF07C008D39753E0A7559F4
:100D3C0005755A24E536C394115005120C5D8006D6
:100D4C009005BBE0F536E536900079F0E56675F078
:100D5C000A84FF7E008F36E56675F00A84ADF07C60
:100D6C00008D39753E0A755905755A5AE536C39486
:100D7C00115005120C5D80069005F1E0F536E53654
:100D8C00900016F02290008CE0B4016AE56675F0D4
:100D9C000A84FF7E008F36E56675F00A84ADF07C20
:100DAC00008D39753E0A755905755A36E536C3946A
:100DBC00115005120C5D80069005CDE0F536853698
:100DCC004AE56675F00A84FF7E008F36E56675F09D
:100DDC000A84ADF07C008D39753E0A755905755A3B
:100DEC0048E536C394115005120C5D80069005DF62
:100DFC00E0F53685364B22E55E75F00484FF7E0007
:100E0C008F36E55E75F00484ADF07C008D39753E4F
:100E1C0004755901755A00E536C3943F5005120C00
:100E2C005D80069001C5E0F5368536287527009063
:100E3C00005CE075F020A4FFAEF09000D7E08E04CB
:100E4C008F05FF1269A08D369000BFE0D3955E50E0
:100E5C0003020F099000E3E0D3955E4010ED900182
:100E6C00C61269E1E0F52A752900020F069000AE62
:100E7C00E0D3955E4043E5369001C61269E1E0F59A
:100E8C0037E5369001E61269E1E0F5389000E3E0D1
:100E9C00F404255EF5399000AEE0FE9000E3E0F43A
:100EAC00042EF53AE537B538058537368003120C34
:100EBC00D785362A7529008041E5369001E61269FE
:100ECC00E1E0F537E5369002061269E1E0F538907D
:100EDC0000AEE0F404255EF5399000BFE0FE900012
:100EEC00AEE0F4042EF53AE537B538058537368093
:100EFC0003120CD785362A752900020FB09000E634
:100F0C00E0D3955E5011E5369002461269E1E0F5AA
:100F1C002A752900020FB09000AFE0D3955E5043C4
:100F2C00E5369002261269E1E0F537E53690024687
:100F3C001269E1E0F5389000AFE0F404255EF53974
:100F4C009000E6E0FE9000AFE0F4042EF53AE537B1
:100F5C00B538058537368003120CD785362A7529A6
:100F6C00008041E5369002061269E1E0F537E5367E
:100F7C009002261269E1E0F5389000BFE0F40425F8
:100F8C005EF5399000AFE0FE9000BFE0F4042EF562
:100F9C003AE537B538058537368003120CD78536D8
:100FAC002A752900229000F7E0F53B753E11755922
:100FBC0002755A00AE51AF52E53B75F00FA4FDAC73
:100FCC00F0EDD39FEC9E4021E53B8E048F05FF1284
:100FDC0069A0ED75F010A4FFAEF0E55E75F011841C
:100FEC00FD7C00ED2FF53C800EE55E75F01184FF65
:100FFC007E00EF24F0F53C853C36E55E75F01184FF
:10100C00AFF07E008F39120C5D85363DAE51AF527C
:10101C009000F7E075F00FA4FDACF0EDD39FEC9EC3
:10102C004028755902755A10853C36120C5D853D69
:10103C0037853638AE51AF52E53B8E048F05FF1223
:10104C0069CB8D39853B3A120CD78536287527002C
:10105C00752A64752900229000F7E0F53B753E1166
:10106C00755902755A00AE51AF52E53B75F00FA49D
:10107C00FDACF0EDD39FEC9E4021E53B8E048F053B
:10108C00FF1269A0ED75F010A4FFAEF0E56075F0ED
:10109C001184FD7C00ED2FF53C800EE56075F011A0
:1010AC0084FF7E00EF24F0F53C853C36E56075F05E
:1010BC001184AFF07E008F39120C5D85363DAE5138
:1010CC00AF529000F7E075F00FA4FDACF0EDD39F9C
:1010DC00EC9E4028755902755A10853C36120C5DF1
:1010EC00853D37853638AE51AF52E53B8E048F05C2
:1010FC00FF1269CB8D39853B3A120CD78536287592
:10110C002700E56A6017E56AC394FE50109000EB67
:10111C00E0B402099000D9E0D3940B50028017AED2
:10112C0027AF28E56A1269B074E78E048F05FF12A9
:10113C0069A08C278D289000C1E0B40453E55E753E
:10114C00F00484FF7E008F36E55E75F00484ADF00C
:10115C007C008D39753E04755901755A00E536C30E
:10116C00943F5005120C5D80069001C5E0F536AE3B
:10117C0027AF28E5361269B074648E048F05FF1210
:10118C0069A0AE27AF28EF2DFDEE3CFC8C278D28F7
:10119C00752A647529002290008CE0B40146E5663E
:1011AC0075F00A84FF7E008F36E56675F00A84AD13
:1011BC00F07C008D39753E0A755905755A00E53677
:1011CC00C394115005120C5D8006900597E0F5361E
:1011DC00AE29AF2AE5362FFF50010E74641269F365
:1011EC008E298F2A90008DE0B40146E56775F00AD0
:1011FC0084FF7E008F36E56775F00A84ADF07C00C5
:10120C008D39753E0A755905755A6CE536C39411BE
:10121C005005120C5D8006900603E0F536AE29AF42
:10122C002AE5362FFF50010E74641269F38E298F54
:10123C002A90009CE0B40249E569C3944175F0051D
:10124C0084FF7E008F36E56975F00584ADF07C0077
:10125C008D39753E05755906755A00E536C39413DC
:10126C005005120C5D8006900699E0F536AE29AF5C
:10127C002AE5362FFF50010E74641269F38E298F04
:10128C002A9000DEE0B402028003021342E55E7590
:10129C00F01584FF7E008F36E55E75F01584ADF099
:1012AC007C008D39753E15755903755AF4E536C3B6
:1012BC00940B5005120C5D8006900485E0F536E524
:1012CC003675F0FFA4FFAEF09000DFE08E048F05C2
:1012DC00FF1269A0ED900072F0E56575F078A4FF3F
:1012EC00AEF074FF8E048F05FF1269A08C598D5AD5
:1012FC0074028C068D071200398F36AC59AD5A74B6
:10130C0004FF1269CB8D39753E04755906755A2840
:10131C00E536C3941D5005120C5D80069006CBE09B
:10132C00F536AE29AF2AE5362FFF50010E74641244
:10133C0069F38E298F2A90008BE0B4025DE560750D
:10134C00F064A4FFAEF074081200398E5B8F5C74ED
:10135C00058E048F05FF1269A08D36AE5BAF5C74F1
:10136C00058E048F05FF1269CB8D39753E057559B5
:10137C0005755ADEE536C394135005120C5D8006D4
:10138C00900677E0F536AE29AF2AE5362FFF5001EF
:10139C000E74641269F38E298F2A9000CDE0703C94
:1013AC0090005CE075F00584FF7E008F3690005C49
:1013BC00E075F00584ADF07C008D39753E057559EE
:1013CC0005755AC0E536C3941D5005120C5D800698
:1013DC00900663E0F536E53690007AF022900094A2
:1013EC00E0B401179008B3E0252AFFAE2950010E96
:1013FC009000E8E01269F38E298F2A90010CE0B47A
:10140C00011490010DE0A851B8000495525007E565
:10141C005EC3955F400280139000B6E0252AFFAEB4
:10142C002950010E8E298F2A021818900094E0B4CE
:10143C000306A227B3B3400280509008BCE07010A2
:10144C009008B6E0C39405A851B800069552400226
:10145C0080109000B6E0252AFFAE2950010E8E298F
:10146C008F2A9008BCE0600D9008B6E0A851B80037
:10147C00069552400280109000B6E0252AFFAE2956
:10148C0050010E8E298F2A02181890008EE0B4029B
:10149C00028003021818900091E0602FE566D39447
:1014AC00464028900017E0FEA3E0FF9000CCE075CA
:1014BC00F003A4FDACF0EFD39DEE9C400E9000F039
:1014CC00E0A851B80005D3955250030218189000AB
:1014DC00C1E0B40302800302167C85605A75590082
:1014EC00900098E0A851B800049552500E900099C5
:1014FC00E0A859B80005D3955A5003021679E56057
:10150C0075F002A4FFAEF074158E048F05FF1269FE
:10151C00A08C068D07900616120048FEE0FFEE9098
:10152C000090E0FEEF8E0088F0A4FFAEF074648EA5
:10153C00048F05FF1269A08C598D5A90005CE075E0
:10154C00F018A4FFAEF09000D7E08E048F05FF12C8
:10155C0069A08C068D0790062E120048AE59AF5A22
:10156C00E01269B074648E048F05FF1269A08C5967
:10157C008D5AE564A859B80077D3955A4072E56442
:10158C00C3955AFFE49559FE8E598F5A7428BE00A4
:10159C00039F500C755A28755900740D90005DF01E
:1015AC00AE59AF5A900091E01269B074288E048F36
:1015BC0005FF1269A08C598D5AAE27AF28740A8E7C
:1015CC00048F05FF1269A08D068C07AC59AD5ACF5C
:1015DC00CECF120003740A8E048F05FF1269A08C03
:1015EC00598D5AAE27AF281269FB8E278F28807D24
:1015FC00E564A859B80004955A5072AE59AF5AE533
:10160C00641269F38E598F5A7428BE00039F500CD4
:10161C00755A28755900740D90005DF0AE59AF5A8B
:10162C00900091E01269B074288E048F05FF126946
:10163C00A08C598D5AAE27AF28740A8E048F05FFE3
:10164C001269A08D068C07AC59AD5ACFCECF1200C3
:10165C0003740A8E048F05FF1269A08C598D5AAE43
:10166C0027AF28EF2DFDEE3CFC8C278D2802181897
:10167C009000D9E0855EF0A4FFAEF074051269B05D
:10168C0074071200398E598F5A900098E0A851B8FF
:10169C00000495525012900099E075F002A4FDAC34
:1016AC00F0EFC39DEE9C4003021818E55E75F00B3D
:1016BC0084FF7E00900616120048FEE0FFEE9000BC
:1016CC0090E0FEEF8E0088F0A4FFAEF074648E0400
:1016DC008F05FF1269A08C598D5A90005CE075F053
:1016EC0018A4FFAEF09000D7E08E048F05FF1269AE
:1016FC00A08C068D0790062E120048AE59AF5AE00A
:10170C001269B074648E048F05FF1269A08C598D18
:10171C005AE564A859B80077D3955A4072E564C36A
:10172C00955AFFE49559FE8E598F5A7428BE0003C2
:10173C009F500C755A28755900740D90005DF0AED1
:10174C0059AF5A900091E01269B074288E048F053D
:10175C00FF1269A08C598D5AAE27AF28740A8E04DB
:10176C008F05FF1269A08D068C07AC59AD5ACFCEF0
:10177C00CF120003740A8E048F05FF1269A08C59D6
:10178C008D5AAE27AF281269FB8E278F28807DE5F6
:10179C0064A859B80004955A5072AE59AF5AE56412
:1017AC001269F38E598F5A7428BE00039F500C7522
:1017BC005A28755900740D90005DF0AE59AF5A90CF
:1017CC000091E01269B074288E048F05FF1269A095
:1017DC008C598D5AAE27AF28740A8E048F05FF12D0
:1017EC0069A08D068C07AC59AD5ACFCECF12000331
:1017FC00740A8E048F05FF1269A08C598D5AAE277E
:10180C00AF28EF2DFDEE3CFC8C278D28229000ECB0
:10181C00E0B4026AE55E75F00884FF7E008F36E561
:10182C005E75F00884ADF07C008D39753E087559F5
:10183C0001755AE0E536C3943F5005120C5D8006E5
:10184C00900285E0F53685362C752B00AE2BAF2C2F
:10185C00AC29AD2A12000374648E048F05FF126943
:10186C00A08C2B8D2C900089E08C068D071269B012
:10187C0074648E048F05FF1269A08C2B8D2CAE27FF
:10188C00AF28AC29AD2A12000374648E048F05FFB7
:10189C001269A08C278D28900089E08C068D071288
:1018AC0069B074648E048F05FF1269A08C278D2893
:1018BC00A203401DAE51AF527405BE00039F5002EF
:1018CC00D203E560D394CC4008D201741190005D32
:1018DC00F09000EBE0B402089000D9E0640B6002D9
:1018EC008035AE27AF28E56A1269B074E78E048F95
:1018FC0005FF1269A08C278D289000ECE0B402172C
:10190C00AE2BAF2CE56A1269B074E78E048F05FF1D
:10191C001269A08C2B8D2C9000ABE05402601B90B4
:10192C0000A2E0A851B80012D39552400DA203B307
:10193C00B35007E560C3949A40028028AE33AF34AD
:10194C009000A0E075F002A4FDACF0EF2DFDEE3C94
:10195C00FC74022DFD50010CE560BC0007D39D40CA
:10196C0003754201856034753300E5427003021A39
:10197C005C9000FEE0C395425003021A4E90010E9B
:10198C00E0C394025076E56675F00A84FF7E009001
:10199C000586120048E0F55A755900AE59AF5A90B9
:1019AC0000A1E01269B074648E048F05FF1269A067
:1019BC008C5B8D5C9000FEE004C395428C068D0719
:1019CC001269B09000FEE08E048F05FF1269A08CA6
:1019DC005B8D5CAE27AF28EF2DFDEE3CFC8C278D8C
:1019EC00289000ECE0B40212AE2BAF2CAA5BAB5CDF
:1019FC00EF2BFBEE3AFA8A2B8B2C80469000FEE004
:101A0C0004C39542854AF0A4FFAEF09000FEE08E30
:101A1C00048F05FF1269A08C5B8D5CAE27AF28EF9D
:101A2C002DFDEE3CFC8C278D289000ECE0B40212CE
:101A3C00AE2BAF2CAA5BAB5CEF2BFBEE3AFA8A2BEE
:101A4C008B2C05429000FEE0C3954250037542007A
:101A5C009000ABE05401601B90009FE0A851B800CF
:101A6C0012D39552400DA203B3B35007E55EC39455
:101A7C00CC4002802590009DE075F003A4FFAEF0F1
:101A8C00E53F2FFF50010E74032FFF50010EE55E52
:101A9C00BE0007D39F4003754301855E3FE543704D
:101AAC0003021B8F9000FFE0C395435003021B8180
:101ABC0090010EE0C394025076E56675F00A84FF3F
:101ACC007E00900586120048E0F55A755900AE5913
:101ADC00AF5A90009EE01269B074648E048F05FFBB
:101AEC001269A08C5B8D5C9000FFE004C395438C65
:101AFC00068D071269B09000FFE08E048F05FF126F
:101B0C0069A08C5B8D5CAE27AF28EF2DFDEE3CFC05
:101B1C008C278D289000ECE0B40212AE2BAF2CAACF
:101B2C005BAB5CEF2BFBEE3AFA8A2B8B2C8046904E
:101B3C0000FFE004C39543854BF0A4FFAEF090008A
:101B4C00FFE08E048F05FF1269A08C5B8D5CAE27C5
:101B5C00AF28EF2DFDEE3CFC8C278D289000ECE09F
:101B6C00B40212AE2BAF2CAA5BAB5CEF2BFBEE3AA4
:101B7C00FA8A2B8B2C05439000FFE0C3954350034E
:101B8C00754300900101E02528FFAE2750010E8E11
:101B9C00278F289000B0E0A827B80004952850099A
:101BAC009000B0E0F5287527009000ECE0B4020D31
:101BBC009000B0E0A82BB80006952C40028009904C
:101BCC0000B0E0F52C752B00229000ECE0B4010283
:101BDC008003021CE0A203B35003021CDE9000B78A
:101BEC00E0B40168AE27AF28AC51AD5212000374BB
:101BFC003C8E048F05FF1269A09000C7E0BC00105A
:101C0C009D400D9000C9E0A827B80004952850020B
:101C1C00D202AE27AF28AC51AD52120003743C8EE9
:101C2C00048F05FF1269A09000C7E0C3940ABC00A2
:101C3C0015D39D40119000C9E0C39405A827B800A6
:101C4C0005D3952850028002C2028068AE27AF28C7
:101C5C00AC51AD5212000374788E048F05FF1269DB
:101C6C00A09000C7E0BC00109D400D9000C9E0A8FA
:101C7C0027B8000495285004D2028038AE27AF282C
:101C8C00AC51AD5212000374788E048F05FF1269AB
:101C9C00A09000C7E0C3940ABC0015D39D401190DE
:101CAC0000C9E0C39405A827B80005D395285002B5
:101CBC008002C202A202B34019AE27AF289000C81E
:101CCC00E01269B074648E048F05FF1269A08C2732
:101CDC008D288002C202A200B34006A201B3B35009
:101CEC000990001FE4F0A3F08024AE27AF28740005
:101CFC00D39F74019E400C90001FE527F0A3E528AC
:101D0C00F0800B74FF90001FF8E4F0E8A3F0900053
:101D1C00B7E0B4011AAE27AF2874021269B08E274F
:101D2C008F28AE2BAF2C74021269B08E2B8F2C9097
:101D3C0000CEE0C394034009900082E0C3940250AB
:101D4C0035AE27AF28745E1269B0740A8E048F0505
:101D5C00FF1269A08C278D289000ECE0B40217AE1E
:101D6C002BAF2C745E1269B0740A8E048F05FF12AF
:101D7C0069A08C2B8D2CAE27AF287402BE000AD321
:101D8C009F4006752802752700AE2BAF2C7402BE3F
:101D9C00000AD39F4006752C02752B0090001DE5A0
:101DAC0027F0A3E528F02290005CE09003861269EE
:101DBC00E1E0F54075416490005CE0FE9000C2E00B
:101DCC00D39E4037E55E75F00884FF7E008F36E5C4
:101DDC005E75F00884ADF07C008D39753E08755940
:101DEC0003755A96E536C3941F5005120C5D800698
:101DFC0090043BE0F5368536418035E55E75F0089C
:101E0C0084FF7E008F36E55E75F00884ADF07C00B3
:101E1C008D39753E08755903755AB6E536C3941F4E
:101E2C005005120C5D800690045BE0F5368536415A
:101E3C00229000F8E0F53B753E11755904755A0077
:101E4C00AE51AF52E53B75F00FA4FDACF0EDD39F56
:101E5C00EC9E4021E53B8E048F05FF1269A0ED75C9
:101E6C00F010A4FFAEF0E55E75F01184FD7C00ED82
:101E7C002FF53C800EE55E75F01184FF7E00EF249B
:101E8C00F0F53C853C36E55E75F01184AFF07E00D4
:101E9C008F39120C5D85363DAE51AF529000F8E093
:101EAC0075F00FA4FDACF0EDD39FEC9E4028755956
:101EBC0004755A10853C36120C5D853D37853638D5
:101ECC00AE51AF52E53B8E048F05FF1269CB8D39B5
:101EDC00853B3A120CD7853640754164229000F848
:101EEC00E0F53B753E11755904755A00AE51AF5271
:101EFC00E53B75F00FA4FDACF0EDD39FEC9E4021BB
:101F0C00E53B8E048F05FF1269A0ED75F010A4FF60
:101F1C00AEF0E56075F01184FD7C00ED2FF53C8092
:101F2C000EE56075F01184FF7E00EF24F0F53C8522
:101F3C003C36E56075F01184AFF07E008F39120CE1
:101F4C005D85363DAE51AF529000F8E075F00FA4B0
:101F5C00FDACF0EDD39FEC9E4028755904755A10DA
:101F6C00853C36120C5D853D37853638AE51AF5207
:101F7C00E53B8E048F05FF1269CB8D39853B3A12F8
:101F8C000CD78536407541649000F3E0B404799029
:101F9C00005CE0FE9000C2E0D39E4037E55E75F039
:101FAC000884FF7E008F36E55E75F00884ADF07C0A
:101FBC00008D39753E08755903755A96E536C394EC
:101FCC001F5005120C5D800690043BE0F5368536FB
:101FDC00418035E55E75F00884FF7E008F36E55E46
:101FEC0075F00884ADF07C008D39753E0875590389
:101FFC00755AB6E536C3941F5005120C5D800690D9
:10200C00045BE0F5368536412290008CE0B4013B50
:10201C00E56675F00A84FF7E008F36E56675F00A7A
:10202C0084ADF07C008D39753E0A755905755A12D0
:10203C00E536C394115005120C5D80069005A9E09D
:10204C00F536E5412536C39464F54190008DE0B436
:10205C00013BE56775F00A84FF7E008F36E56775F6
:10206C00F00A84ADF07C008D39753E0A7559057502
:10207C005A7EE536C394115005120C5D800690060D
:10208C0015E0F536E5412536C39464F541E5402568
:10209C0041F535900094E0B402109008B2E025357B
:1020AC00FE9000E8E0F4042EF5359000EBE0D394BC
:1020BC00014040E56AC394E7501D74E7C3956AFE7E
:1020CC009008B4E08E00F5F0E884FF7E008F36E5D2
:1020DC00352536F535801CE56AC394E7FE9008B4C7
:1020EC00E08E00F5F0E884FF7E008F36E535C39571
:1020FC0036F535A2034006E5402464F535E535D3C5
:10210C0094644009E535C39464F535800375350056
:10211C009000C4E0C3953550069000C4E0F535221C
:10212C00D200900078E0A851B800049552503E902F
:10213C000078E0A851B800049552500375350F9003
:10214C000078E004A851B800049552500375350787
:10215C00900078E02402A851B8000495525002C2B5
:10216C0000900078E06006740990005DF0C22E7E4D
:10217C00017F009000CAE01269B09000D9E08E0493
:10218C008F05FF1269A0E55EBC0017D39D4013902C
:10219C0000D3E0B40204D22E8002C200740A900074
:1021AC005DF090008CE0B401099000CBE0C3956623
:1021BC00400280159000DDE0A851B8000495525003
:1021CC0002C200740B90005DF090008CE0B401072B
:1021DC00E566C394644002801D900123E0600D907D
:1021EC000123E0A851B80006955240028008C200B5
:1021FC00740B90005DF0A200400375350090010C4B
:10220C00E0B4011490010DE0A851B80004955250AF
:10221C0007E55EC3955F400280209000B5E0D39443
:10222C001D400B9000B5E0C3941EF5358003753549
:10223C0000741590005DF002231D900094E0B4032F
:10224C0006A227B3B3400302231D9008B6E0C39443
:10225C0005A851B80004955250069008BCE06002E5
:10226C00801D9000B5E0D3941D400B9000B5E0C3E9
:10227C00941EF5358003753500740C90005DF0905C
:10228C0008B6E0A851B80004955250069008BCE07E
:10229C007002801D9000B5E0D3941D400B9000B5EA
:1022AC00E0C3941EF5358003753500740C90005D09
:1022BC00F09008B6E0A851B8000495525031900047
:1022CC00D3E0B40228D22E9008BBE0FE9008BCE00C
:1022DC00D39E50069008BCE0700280099008BBE4C5
:1022EC00F0C22E80069008BBE004F08002C2009081
:1022FC0008B6E02405A851B800049552501390007C
:10230C00D3E0B4020A9008BCE07002D22E8002C264
:10231C0000A22DB3401D9000B5E0D3941D400B904E
:10232C0000B5E0C3941EF53580037535007410902C
:10233C00005DF085356B9000B5E0D3941D4018908E
:10234C000083E02535FE90005CE075F01E84FC7F78
:10235C0000EE2CF535804990005DE0640C600F9028
:10236C00005DE06410600790005DE0B4151690000D
:10237C0083E0FE90005CE075F01E84FC7F00EE2C88
:10238C00F535801C900085E02535FE900083E02E0D
:10239C00FE90005CE075F01E84FC7F00EE2CF535A1
:1023AC002290005CE075F00584FF7E008F36900073
:1023BC005CE075F00584ADF07C008D39753E0575DB
:1023CC005903755AD69000D7E01475F00584FF7E3A
:1023DC0000E536BE00039F5005120C5D800BE53600
:1023EC0090045C1269E1E0F536E5369008B5F090A2
:1023FC0008B5E0FE9000C6E0C39E50089000C6E011
:10240C009008B5F022E56675F00A84FF7E00900511
:10241C0086120048E0F545E545D394644010E54547
:10242C00C3946475F00F84FF7E008F45800375455F
:10243C00009000A9E02545F54522E56675F00A8473
:10244C00FF7E00900586120048E0C39469505590B9
:10245C0000F3E0C394035026900888E0FEA3E0FF4D
:10246C007404120039E55E1269B0740F8E048F0586
:10247C00FF1269A0900886ECF0A3EDF08024900880
:10248C0088E0FEA3E0FF7404120039E5601269B025
:10249C00740F8E048F05FF1269A0900886ECF0A3D0
:1024AC00EDF0800F900888E0F8A3E0900886C8F063
:1024BC00A3C8F0A203401A900888E0FEA3E0FF74C2
:1024CC00031269B07401120039900886EEF0A3EF84
:1024DC00F0900886E0FEA3E0FF90088CE0FCA3E0FF
:1024EC00FDEDD39FEC9E400F90088CE0F8A3E0909C
:1024FC000886C8F0A3C8F090009CE0B40262E569BD
:10250C00C3944175F00584FF7E008F36E56975F044
:10251C000584ADF07C008D39753E05755906755AEC
:10252C0014E536C394175005120C5D80069006AD69
:10253C00E0F536900886E0FEA3E0FF740A8E048F67
:10254C0005FF1269A0E5368C068D071269B0740A76
:10255C008E048F05FF1269A0900886ECF0A3EDF0B5
:10256C0022E50875F004A4FFAEF09006C9120048ED
:10257C00E09032A1F8282873804C855272804790E5
:10258C0000D9E0855EF0A4FFAEF074081200398F1C
:10259C00728033856072802E8566728029856772A1
:1025AC008024856872801F856972801A856A7280A2
:1025BC00158565728010856472800B856B72800640
:0625CC00900020E0F57212
:1032A10002258402258602258B02259F0225A40280
:1032B10025A90225AE0225B30225B80225BD0225A6
:0732C100C20225C70225CC63
:1025D200E50875F004A4FFAEF09006CA120048E5C3
:1025E2000875F004A4FFAEF0E0FC9006CB120048A0
:1025F200ECFEE0FFEEC39F40030226DAE50875F029
:1026020004A4FFAEF09006C9120048E0B40441E50C
:102612000875F004A4FFAEF09006CB120048E0C3A8
:102622009572500AE508F50CD3922F123FADE508DA
:1026320075F004A4FFAEF09006CA120048E0D395EC
:1026420072400AE508F50CC3922F123FAD0226D85C
:10265200E50875F004A4FFAEF09006CA120048E047
:10266200C395725015E50875F004A4FFAEF090060C
:10267200CB120048E0D395725002800AE508F50CAF
:10268200D3922F123FADE50875F004A4FFAEF0908F
:1026920006CA120048E0D395725015E50875F00499
:1026A200A4FFAEF09006CB120048E0C39572500A28
:1026B200E508F50CC3922F123FAD9006D1E0B401AC
:1026C200099000E5E0D395605002800A7402F50C8F
:1026D200C3922F123FAD806AE50875F004A4FFAEE5
:1026E200F09006CA120048E0D395724015E50875CD
:1026F200F004A4FFAEF09006CB120048E0C395723E
:102702004002800AE508F50CC3922F123FADE5089E
:1027120075F004A4FFAEF09006CA120048E0C3951B
:10272200724015E50875F004A4FFAEF09006CB12D6
:102732000048E0D39572400AE508F50CD3922F12B7
:102742003FAD22AE2DAF2E74C9BE000CD39F400800
:10275200782D126A0302285F752E01752D00AE5185
:10276200AF52E545BE000DD39F40099000BBE0D3B8
:10277200954640028023754600E545C39552F572A1
:102782009000BEE0D395444008E5442572F54480AC
:10279200069000BEE0F54480020546900097E0D323
:1027A2009560401CE55EC3955F4015AE51AF52E5A2
:1027B20045BE00039F50099000BCE0D395474002FC
:1027C200806E9008B7E0A851B80004955250037586
:1027D20049009008B7E0A851B8000BD395524006C3
:1027E200E5529008B7F0E5497041E552C39545F5C9
:1027F20072E572D3940540037572059000BDE0C383
:1028020095445007E572C3954440028009E544C3EC
:102812009572F54480069000BDE0F5449000BDE05D
:10282200D3954440069000BDE0F544754700800210
:102832000547E5497016900097E0C39560500DE595
:10284200452405A851B8000695524002800F900019
:10285200AAE0F54475490174789008B7F022AE2DCC
:10286200AF2E74E9D39F74039E4008782D126A0339
:10287200022A06752E01752D00754432A228402ABF
:102882007544199000AAE075F002A4FFAEF0E54687
:10289200BE0006D39F4002D22805467549037478CC
:1028A2009008B7F07548000229EDAE51AF52E545E8
:1028B2006F4E70030229EDE545BE000DD39F40091E
:1028C2009000BBE0D395464002800F754600E54973
:1028D200C394035003754419800DE545C39552F521
:1028E20072E5462572F546900097E0D39560400E5A
:1028F2009008B7E0A851B80007D395524002800C67
:1029020005489000AAE0B54803754900E549B403BB
:1029120006A203B3B34002800A0548E548B43C036B
:10292200754902E549B402299008B7E0A851B800F8
:102932000ED395524009E5529008B7F075480090C1
:102942000097E0C39560500975480074789008B705
:10295200F0E549705A900097E0D39560401CE55E1F
:10296200C3955F4015AE51AF52E545BE00039F507F
:10297200099000BCE0D39547400280087547007576
:10298200444B8028E552C39545F572E572D3940510
:102992004003757205900097E0D395604008E547C3
:1029A2002572F5478006E5472406F547754800E598
:1029B200497016900097E0C39560500DE5452405D7
:1029C200A851B80006955240028003754901E549B5
:1029D200B4011875441905489000AAE0B548067577
:1029E200490275480074789008B7F0A201B3400319
:1029F200754432E54475F00AA4FFAEF090088EEEFD
:102A0200F0A3EFF022E56E9032C8F8282873900008
:102A12008FE07003022C449000C5E0B401028003F1
:102A2200022B4F90005AE0655D6009E55245516006
:102A320003022B4C7E017F00E5BE1269B0E5BD2F7B
:102A4200FF50010E8E598F5A74101269B0900077A0
:102A5200E08E048F05FF1269A0900892ECF0A3EDBE
:102A6200F0E56A600FE56AC394FE50089000EBE05F
:102A72006402600280649000D9E0B40B1F90089257
:102A8200E0FEA3E0FF74E71269B0E56A8E048F05E9
:102A9200FF1269A0900892ECF0A3EDF09000D9E04B
:102AA200D3940B40089000C1E064046002802B9034
:102AB2000892E0FEA3E0FF900896E0FCA3E0FDEFA1
:102AC200D39DEE9C400D1269FB900892EEF0A3EFAD
:102AD200F08007900892E4F0A3F090008FE0B40237
:102AE20027900894E0FEA3E0FF900892E0FCA3E0A8
:102AF200FDEF2DFDEE3CFC74018C068D07120039B2
:102B0200900892EEF0A3EFF0900892E0FEA3E0FFAF
:102B1200900894E0FCA3E0FDEDD39FEC9E4004D22C
:102B22002C8002B22C900892E0F8A3E0900894C89E
:102B3200F0A3C8F09000C1E064016006A22CB3B318
:102B420040028006900893E0F55E022C42D22C7E71
:102B5200017F00E5BE1269B0E5BD2FFF50010E8E68
:102B6200598F5A74101269B0900077E08E048F0565
:102B7200FF1269A0900892ECF0A3EDF0E56A600FF5
:102B8200E56AC394FE50089000EBE06402600280A4
:102B9200649000D9E0B40B1F900892E0FEA3E0FF1E
:102BA20074E71269B0E56A8E048F05FF1269A0907E
:102BB2000892ECF0A3EDF09000D9E0D3940B40081A
:102BC2009000C1E064046002802B900892E0FEA3B2
:102BD200E0FF900896E0FCA3E0FDEFD39DEE9C4061
:102BE2000D1269FB900892EEF0A3EFF080079008B7
:102BF20092E4F0A3F090008FE0B40227900894E0F2
:102C0200FEA3E0FF900892E0FCA3E0FDEF2DFDEEB5
:102C12003CFC74018C068D07120039900892EEF08C
:102C2200A3EFF0900892E0F8A3E0900894C8F0A314
:102C3200C8F09000C1E064016006900893E0F55E80
:102C42008003755E0090008BE07006756E01022AAB
:102C52000775BB1802327B90008BE07003022DCA0D
:102C62007E017F00E5BE1269B0E5BD2FFF50010E67
:102C72008E598F5A9000D1E0B4010F7E0F7FFFACC6
:102C820059AD5A1269FB8E598F5A9000F6E0B40280
:102C920045AE59AF5A900029E0FCA3E0FDEDD39F69
:102CA200EC9E400A900029E559F0A3E55AF0AE598E
:102CB200AF5A90002BE0FCA3E0FDEFD39DEE9C40C9
:102CC2000A90002BE559F0A3E55AF0AE59AF5A74B9
:102CD200041200398F609000F6E0704CAE59AF5A82
:102CE200900029E0FCA3E0FDEFD39DEE9C40091289
:102CF20069FB8E598F5A8006755A00755900AE5974
:102D0200AF5A74101269B0900074E08E048F05FF00
:102D12001269A08C598D5A74FFBC0009D39D4005DD
:102D2200855A6080037560FE9000C1E0B4010280A4
:102D320003022DC8A203B3B3500E900095E0A85130
:102D4200B80005D39552500280719000D2E08560A0
:102D5200F0A4FFAEF074648E048F05FF1269A08C9C
:102D6200598D5AE56A6016E56AC394FE500F9000C9
:102D7200EBE0B402089000D9E0640B60028017AE69
:102D820059AF5A74E71269B0E56A8E048F05FF12D3
:102D920069A08C598D5AAE59AF5A900892E0FCA3A3
:102DA200E0FDEDD39FEC9E4005855A5E800BA22C80
:102DB200B34006900893E0F55E800BA22CB3400668
:102DC200900893E0F55E800375600090008EE070DD
:102DD20006756E02022A0775BB1902327B90008EBD
:102DE200E07003022E7FE55DD395504003022E7DF5
:102DF200900027E0FEA3E0FFE5641269F39000274C
:102E0200EEF0A3EFF07E017F00E5BE1269B0E5BDF2
:102E12002FFF50010E8E598F5A9000FBE0701374F1
:102E22000A1269B074518E048F05FF1269A08D6475
:102E32008019AE59AF5A740A1269B08F048E057E9A
:102E4200017F95CDCCCD12689E8F64E564D39464E6
:102E52004003756464900027E0FEA3E0FFE5642F61
:102E6200FF50010E900027EEF0A3EFF0900092E0E9
:102E7200048E048F05FF1269A08D6480037564328D
:102E82009000DEE07006756E03022A0775BB13021E
:102E9200327B9000DEE0604A7E017F00E5BE12696F
:102EA200B0E5BD2FFF50010E8E598F5A74041200E7
:102EB200398F659000E0E08565F0A4FDACF07464A4
:102EC200FF1269A08D659000DFE08565F0A4FFAE7A
:102ED200F074FF8E048F05FF1269A0ED900073F06D
:102EE200800375650090008CE07006756E04022AFE
:102EF2000775BB1702327B90008CE0B4010280039D
:102F0200022F8D7E017F00E5BE1269B0E5BD2FFF65
:102F120050010E8E598F5A9008B8E060199008B887
:102F2200E0149063D812008CE493FC740193FDEDDD
:102F3200C39FEC9E400280069008B8E014F090080F
:102F4200B8E0C394B3501DAE59AF5A9008B8E0042C
:102F52009063D812008CE493FC740193FDEFC39D3F
:102F6200EE9C400280069008B8E004F09008B8E0B9
:102F7200FE9000B2E08E0088F0A4FFAEF074648E82
:102F8200048F05FF1269A08D6680037566009000AC
:102F92008DE07006756E05022A0775BB1602327B3C
:102FA20090008DE0B4010280030230367E017F0082
:102FB200E5BE1269B0E5BD2FFF50010E8E598F5A42
:102FC2009008B9E060199008B9E0149065421200C7
:102FD2008CE493FC740193FDEDC39FEC9E40028050
:102FE200069008B9E014F09008B9E0C394B3501DFC
:102FF200AE59AF5A9008B9E00490654212008CE4D1
:1030020093FC740193FDEFC39DEE9C4002800690F9
:1030120008B9E004F09008B9E0FE9000B8E08E0034
:1030220088F0A4FFAEF074648E048F05FF1269A0CD
:103032008D67800375670075BB1F02327B7E017F3F
:1030420000E5BE1269B0E5BD2FFF50010E8E598F0B
:103052005A74091269B074E68E048F05FF1269A0D2
:103062008D69900094E07006756E07022A0775BBA1
:103072001502327B900094E070030231C77E017F1B
:1030820000E5BE1269B0E5BD2FFF50010E8E598FCB
:103092005A74041200398F68900094E0B4011590BC
:1030A20000E8E08568F0A4FFAEF07407120039EF83
:1030B2009008B3F0900094E0B402159000E8E08527
:1030C20068F0A4FFAEF07407120039EF9008B2F076
:1030D200900094E0B4030280030231AA9000D5E08C
:1030E2007052E568C39419500FD2279000B4E09053
:1030F20008B6F09008BAE4F0E568D394644004A2FC
:10310200274002802D9008BAE004F09008BAE0FE51
:10311200900127E0B5060B9008B6E004F09008BADB
:10312200E4F09008B6E064966006900127E0700231
:10313200C22780639000B4E070349000E8E08568B4
:10314200F0A4FFAEF074FF8E048F05FF1269A0EDAC
:103152009008B6F0AE51AF52741EBE0006D39F4027
:1031620002D227E560D394E54002C2278029E568B0
:10317200C3940A500DAE51AF52741EBE0004D39FC9
:1031820050028002D227E560D394E54002C2279024
:1031920000B4E09008B6F09008B6E0C3940550067B
:1031A20074059008B6F0C22D900094E0B40414E5C2
:1031B20068C394195002D22DE568D394324002C2FA
:1031C2002DC22780037568009000EBE07006756ED3
:1031D20008022A0775BB1402327B9000EBE07003F1
:1031E20002326A7E017F00E5BE1269B0E5BD2FFFA3
:1031F20050010E8E598F5A900110E07025EFD39432
:1032020021EE940E4005756AFF8015AE59AF5A74CF
:10321200101269B074E38E048F05FF1269A08D6AE3
:103222008027AE59AF5AEFD39449EE940640057504
:103232006AFF8015AE59AF5A74101269B074658E68
:10324200048F05FF1269A08D6AE56A75F00BA4FF71
:10325200AEF09000D9E08E048F05FF1269A09008AD
:1032620096ECF0A3EDF08003756A0090008FE060A9
:093272000575BB1A800375BB1839
:1032C800022A10022C59022DDF022E94022EF90236
:0B32D8002FA202303F0230760231DCF2
:05327B00056ED2EC22FB
:0969E1002582F582500205832293
:0F008C0025E050020583258250020583F582226C
:10697F00EF2F500205832582F582E5833E2EF583A6
:01698F0022E5
:1069F300CFC39FFF50011E22C3EF9DFFEE9CFE22DB
:086A03000806B6000218062285
:0D69BE00A3E004F070061269D7E004F02297
:086A0B000816B6FF021816225E
:0E003900048007C3CE13CECF13CFD5E0F6223E
:10689E00BC000FBE0008ED8FF084FFADF022E4FEC9
:1068AE00FF22BE000DEF60FE54F0606F20E7030282
:1068BE006954EAC0E0EBC0E078017A0075F001EEB1
:1068CE0020E710EF25E0FFEE33FE0AC5F023C5F0FA
:1068DE0030E7F0EA5407F9096A7A007B0060010894
:1068EE00C3EC9E40167004ED9F4010ED9FFDEC9E94
:1068FE00FCE5F0CA4ACA03F5F08005E5F003F5F0B1
:10690E00C3EE13FEEF13FFD9D77908CACBCAD8D07E
:10691E00EAFEEBFFD0E0FBD0E0FA22EC8FF084FC35
:10692E00ED54F045F0C48FF084FEEDC454F045F004
:10693E00C48FF084FDEEC4FE54F02DFFEE540F3CD8
:10694E00FEADF07C0022790078008FF0EC7E0820FE
:10695E00E70DC3CD33CD33C933C9C833C8DEF08498
:10696E0049F9E5F08FF0BE00E6FD7C00E9FFE8FE98
:01697E0022F6
:0E69B000F88FF0A4FFE5F0CE88F0A42EFE22B2
:10000300EF8DF0A4F9A8F0EF8CF0A428F8EE8DF0B2
:06001300A428FEE9FF2213
:10699000600D782B02699A007830D8FED5E0F82295
:1069A000EEC0E07E0012689EEFFDEEFCD0E0FE221D
:0C69CB00EEC0E07E0012689ED0E0FE22CC
:03001B0002001EC2
:0300530002005652
:03009B00020071EF
:030000000269EAA8
:0969EA0075817475D00002422F82
:0B004800E5822FF582E5833EF5832260
:0A69D7000582D58202158315822285
:10001E00C0E0C0F0C083C082C0D075D000124135A0
:0B002E00D0D0D082D083D0F0D0E032E0
:10005600C0E0C0F0C083C082C0D075D00012413865
:10006600D0D0D082D083D0F0D0E032C0E0C0F0C093
:1000760083C082C0D075D0001241E2D0D0D082D0E9
:0600860083D0F0D0E0324F
:00000001FF
